:020000040000FA
:2000000000000000000000000000000000000000000000000000000000000000800044001C
:2000200002043E060000000000000000000000000000000000000000000000000000000076
:200040000000000000000000000000003E0B000000003E0B000000003E0B000000003E0B7C
:20006000000000003E0B000000003E0B000000003E0B000000003E0B000000003E0B000013
:2000800000003E0B000000003E0B000000003E0B000000003E0B000000003E0B00000000F3
:2000A0003E0B000000003E0B000000003E0B000000003E0B000000003E0B000000003E0B8A
:2000C000000000003E0B000000003E0B000000003E0B000000003E0B0000000000000000FC
:2000E00000000000000000000000000000000000000000003E0B000000003E0B000000006E
:200100003E0B000000003E0B000000003E0B000000003E0B000000003E0B000000003E0B29
:20012000000000003E0B000000003E0B000000003E0B000000003E0B000000003E0B000052
:2001400000003E0B000000003E0B000000003E0B000000003E0B000000003E0B0000000032
:200160003E0B000000003E0B000000003E0B000000003E0B000000003E0B000000003E0BC9
:200180001C0000000210000000043E0B00000000060F1C000000061100000000300F00005D
:2001A0000000340F00000000370F00000000380F000000003C0F000000003F0F00000000D6
:2001C000250F01000000260F000000002D0F010000002E0F000000000A10A01C02003E0124
:2001E000BA0130003E02AA0131003E02000000000A11000001000D14001800000B14210221
:2002000000000E0F060000000F0F03000000001000C810003E02410000002D1146000000AD
:200220002E11040002001F0FC2000200BE0602A000003E015C000200200645000000031105
:20024000C2000200BE06201002003E01C2000200BE06001002003E0116000000200700008F
:20026000DBB1090FBB0830003E02000000000B1100000200010F00010000020F2F0417001D
:200280003E01410000002E1104000200140F40000200180F000000001C0F40148285CF7048
:2002A00094FFFF00000E000000804F7604000200000F000000B20F7040000000011142007F
:2002C00000000211470000000411040002043E061C0000000E1100000000800000A0020004
:2002E0003E0103000000000700A002003E01050000002007002000883F7001000000020D41
:2003000000000080BE51600002003E0600A002003E0107000000200700000000DC0F0000AE
:200320000000DD0F002000883F7001000000020D000080EDBE51600002003E0600A00200A6
:200340003E01080000002007000000883F7004000000020DC2000204BE0600000000000059
:2003600000000000000000008081BE51600002003E0600A002003E010800000020070000B7
:2003800000883F7004000000020DC2000204BE060000000000000000000000000000808186
:2003A000BE51600002003E0600A002003E01080000002007000000883F7004000000020D2E
:2003C000C2000204BE06000000000000000000000000000080EDBE51600002003E0600A0CF
:2003E00002003E01D8FFFF00000700A002003E01D6FFFF00000700A002003E01DAFFFF006A
:20040000000700A002003E0107000000200700000000DC0F00000000DD0F0020008C3F7094
:2004200001000000020D000080EDBF51600002003E0600A002003E01D8FFFF00000700A02B
:2004400002003E01DFFFFF00000700A002003E01E6FFFF00000700A002003E016000020068
:2004600020060000008C3F7004000000020DC2000204BE060000000000000000000000007C
:20048000000080EDBF51600002003E06000000000D10000000000B11400000001F1142004E
:2004A00000002E11470000000F111C0000000E1100000000800004000200DB1200000000E8
:2004C0000D11000000043E0A00000081CF7D20128281DF7D00000000000000000000000054
:2004E0000000000000000000000000000000000000000000000000000000000000000000FC
:200500000000000000000000000000000000000000000000000000000000000000000000DB
:200520000000000000000000000000000000000000000000000000000000000000000000BB
:2005400000000000000000000000000000000000000000000000000000000000000000009B
:2005600000000000000000000000000000000000000000000000000000000000000000007B
:2005800000000000000000000000000000000000000000000000000000000000000000005B
:2005A00000000000000000000000000000000000000000000000000000000000000000003B
:2005C00000000000000000000000000000000000000000000000000000000000000000001B
:2005E0000000000000000000000000000000000000000000000000000000000000000000FB
:2006000000002A06400001000000000002000000000003000000000004000000000005005B
:0A06200000000000060000000000CA
:20062A000E0000000000ED0C00010200030102000206DB0FC940040F042008003E01F91618
:20064A000204BE06308C02000011000000000000B88C02000110010013003E0101800200CA
:20066A000110011008003E010180020000118D8C02000010001002003E011C0102000006D2
:20068A00318C020000102E8C02000410041008003E01140102000206DB0FC940040F04200D
:2006AA0008003E01F9160204BE06318C02000011000000000000B98C0200011001001300D4
:2006CA003E01018002000110011008003E0101800200001101800200001055EB020000116B
:2006EA002A380200001357EB020000112C3802000013918C02000010001002003E013601F4
:20070A00020000068C9D020000100D661900040F004011003E01FEFF0000010F000141000E
:20072A003E0104C018003E01000040003E018C9D02000011E1FFFFFF0C0F0CA00D003E01A9
:20074A00BA8C02000110010013003E0156EB020000112B380200001357EB020001100111B0
:20076A0008003E0157EB020001112C380200001300000000000F001002003E01A401020052
:20078A000006C7000000001000000020010F010004003E014B010200000601000000000F9A
:2007AA00001002003E014601020000064AA10200140F00000000340F1A000000680F0100AA
:2007CA0000001E0E0000000000994B0102003E062DA10200140F00000000340F1D00000065
:2007EA00680F010000001E0E00000000009901000000000F001002003E01750102000006D3
:20080A004AA10200140F00000000340F4BEB0200150F00000000350F203802001C0F0A004C
:20082A000000680F030000001E0E000000003E59000000803E5B000000803F5958EB0200FB
:20084A00150F2D3802001C0F02000000260F020000002D0F08000000680F030000001E0EB5
:20086A00000000003E5900000080BE5B000000807F5902800200150F08000000680F0200BD
:20088A0000001E0E000000003E59000000803E5BC60000000010FFCFFFFF010F01000400BB
:2008AA003E01C600000000114AA10200000F38000000001101000000000F39000000001179
:2008CA001A000000000F3A0000000011C6000000001000300000010FA40102043E06011084
:2008EA0004003E01C600000000112DA10200140F00000000340F41EB0200150F000000004C
:20090A00350F163802001C0F0A000000680F030000001E0E000000003E59000000803E5BAE
:20092A00000000803F5957EB0200150F2C3802001C0F02000000260F020000002D0F08001F
:20094A000000680F030000001E0E000000003E5900000080BE5B000000807F5902800200DB
:20096A00150F08000000680F020000001E0E000000003E59000000803E5B000000003E5955
:20098A0055EB020000112A3802000013000000003E5957EB020000112C380200001300001E
:2009AA0000003E5956EB020000112B3802000013C60000000010FFCFFFFF010F0100040013
:2009CA003E01C600000000112DA10200000F38000000001101000000000F39000000001175
:2009EA001D000000000F3A0000000011C6000000001000300000010F011004003E01C60046
:200A0A000000001100000000000F68EB0200001169EB020000116AEB020000116BEB02001F
:200A2A000011D8E60200140F00000000340F68EB0200150F00000000350F9EA00200081060
:200A4A000C000000080D882804003E59001002003E01BA0102000006CC2C04003E010400CD
:200A6A000000000D153802001C0F000080163E59000000287F0400C8582A012900C8580079
:200A8A003E018C1808003E01000000843E5B2CE30200140F6CEB0200150FA0A002000810FA
:200AAA000C000000080D882804003E59001002003E01CA0102000006CC2C04003E0104005D
:200ACA000000000D153802001C0F000080163E59000000287F0400C8582A012900C8580019
:200AEA003E018C1808003E01000000843E5BF00A0000340F64A10200440F54AC02001410E8
:200B0A00000000283F0454AC02001411FCA00200261068EB0200150F7AED0200160F00005E
:200B2A000000360F9EA00200001004000000000D000000804F71000000803E5D00000000AA
:200B4A003E5B00000080BE59000001008014010202001A06000004008014E00102001A0606
:200B6A00000002008014020202003A0685EB0200160F00000000360F6CEB0200150FA0A0F6
:200B8A0002006810020000001E0E000000023E5B000000823E5D54AC0200011055AC0200D5
:200BAA00011146B70200011047B70200011138D80200011039D8020001117AED0200011035
:200BCA007EED020001117BED020001107FED020001117CED0200011080ED020001117DED2A
:200BEA000200011081ED02000111000002008014FB0102003A0686ED0200011085ED020088
:200C0A00011100000000010F86ED02000111000004008014010202003A0684ED02000110C0
:200C2A0083ED0200011100000000010F84ED02000111000007002014928C020001100A001B
:200C4A000000000F012000003E013A0202000006F00A0000340F56AC0200440F46B7020044
:200C6A001410000000283F0446B702001411FEA00200261000000000000F9FA00200681019
:200C8A00010000001E0E00000080BE5900000000340F00000000000F012000003E011602BC
:200CAA000200200600000000000F340202003E0601000000000F012000003E011B020200E8
:200CCA00200655EB02000010340202003E0602000000000F012000003E012002020020065B
:200CEA0056EB02000010340202003E0603000000000F012000003E0125020200200657EB18
:200D0A0002000010340202003E0604000000000F012000003E0130020200200641EB020040
:200D2A00140F58EB0200150F00000000350F378C02006810020000001E0E000000003E59D7
:200D4A00000000803E5BCE0302003E0605000000000F012000003E01CE030200200641EBC0
:200D6A000200001058EB0200150F00000000350F378C02006810010000001E0E00000080C0
:200D8A003E5BCE0302003E0680EB02000410409402003E0180EB0200041181EB02000410FF
:200DAA00409402003E0181EB020004117AED0200100F00000000300FCAA00200110F00003E
:200DCA000000310FDAA00200120F00000000320FEAA00200130F00000000330F58EB0200B6
:200DEA00150F21ED0200160F00000000360F4CED0200170F00000000370FFAA002002610D2
:200E0A0000000000270FFEA002002D10000000003D0F003002001E0F000000003E0F003489
:200E2A0002001F0F000000003F0F82EB02000310000000000F0F46B702000E109FA002002C
:200E4A000D10F00A0000340F64A10200440F00000004FE5B000000003E5300A082003E5531
:200E6A00000000900F7010A102003E400000008A0F703FC02C003E01760202003006000005
:200E8A00008EEF71CC2C0422012901000000010D00C85822012900C858003E018C1808008C
:200EAA003E01040000008014760202003A060000808EFF71F00A0000340F56AC0200440F85
:200ECA000000008AEF70CC2C04620129000080003E5710A102003E0101000000010D00C8B9
:200EEA005862012900C858003E018C1808003E01000000A87F04000000E87F04F00A00002A
:200F0A00340F56AC0200440F00008085EF700000008AEF70000000303F04000000874F7126
:200F2A0000000002FE5D77BE7F3F000F000080808F7080380E003E01812108003E018F02CA
:200F4A0002000006020000000C0F409402003E014C2C00003E0192020200040600004000B6
:200F6A00001449ED020001101F012C003E01920202043E0649ED0200011100000000040F44
:200F8A00920202003E0640A402003E0192020200220600000000040F000000823E5D00005A
:200FAA0000843E5B0000008ABF70000000283F04000000843E59880413003E01000080006D
:200FCA00FE5F141108003E01000080803E5FF09F02003E01DF2100003E015902020024060B
:200FEA004BED02000010009002003E014BED02000011F00A0000340F56AC0200440F46B7F0
:20100A0002001410000000283F0446B702001411010000008014CE0302003A061000000059
:20102A008014CE0302003A0600000000000F001002003E01810302040006F00A0000340FD2
:20104A0048CD0200440F01000000000F001002003E011A030204000602800200150F0000EA
:20106A000000350F38D802001410000000283F0438D802001411FBA002002610F1FFFFFF89
:20108A000C0F20A10200031082EB02000210000000000F0F9FA0020008102FC02C003E0103
:2010AA00CC020204300600000000040FF09F02003E018A9D020000100D661900040F004021
:2010CA0011003E01FEFF0000010F000141003E0104C018003E01000440003E018A9D020061
:2010EA00041114F001783E021CA00D003E01030413003E0100000082BE5900000000FE5BC1
:20110A00000000823E5B8F2400003E01D5020200040600000080BE59F09F02003E018F20BF
:20112A0000003E01BD02020024060400000080140B0302003A060800000080140B030200E7
:20114A003A06003402001F0FF00A0000340F3AD80200440F58EB0200150FF00A0000360F95
:20116A0048CD0200460F38D802001610F00A0000370F3AD80200470F2AE30200171082EB74
:20118A0002000310000000000F0FEAA00200130F9FA002000D100000008EFF710000008A7E
:2011AA007F713FC02C003E01F20202043006882884003E5710A10206BE5D000000220129B2
:2011CA0001000000010D00C85822012900C858003E018C1808003E0100000000FE5B0810CF
:2011EA0008027F5F000000803E5B0000008A7F71000000283F04000000843E59000000F0F4
:20120A003F04F09F02003E01FD2000003E0107030200220600000006BE5D0000008A7F7186
:20122A00000000283F04000000863E59000000E03E04000000F03F04000000603F04000024
:20124A0000E87F04F09F02003E01FD2000003E01E702020002062AE302001710CE030204ED
:20126A003E06000000E83F042AE30200171138D80200141058EB0200150F02000000020F0C
:20128A00000000000F0F9FA002000D1000000000BE5900008000FE5B011108003E0100007F
:2012AA0080803E5B000000303F04000000603F042F1F00003E01FD2000003E01CE030200B9
:2012CA002206100302003E0638D802001410000000283F0438D802001411FBA002002610D8
:2012EA00F1FFFFFF0C0F20A10200031082EB02000210000000000F0F9FA00200081000000D
:20130A000000FE5B00000080BE59F09F02003E018F2400003E013C03020004062FC02C00AB
:20132A003E0137030204300600000000040FF09F02003E018A9D020000100D661900040F33
:20134A00004011003E01FEFF0000010F000141003E0104C018003E01000440003E018A9DA0
:20136A000200041114F001783E021CA00D003E01030413003E0100000082BE590000008213
:20138A003E5B8F2000003E019B0302000406230302003E06040000008014720302003A0657
:2013AA00080000008014720302003A06003402001F0FF00A0000340F3AD80200440F58EB85
:2013CA000200150FF00A0000360F48CD0200460F38D802001610F00A0000370F3AD80200A6
:2013EA00470F2AE30200171082EB02000310000000000F0FEAA00200130F9FA002000D10AB
:20140A0000000006BE5D0000008A7F71000000283F04000000863E59000000E03E0400007D
:20142A0000F03F04000000603F04000000E87F04F09F02003E01FD2000003E016E030200C2
:20144A0022060000008EFF710000008A7F713FC02C003E01640302043006882884003E570C
:20146A0010A10206BE5D00000022012901000000010D00C85822012900C858003E018C18C4
:20148A0008003E0100000000FE5B081008027F5F000000803E5B0000008A7F7100000028E7
:2014AA003F04000000843E59000000F03F04F09F02003E01FD2000003E014E03020002060A
:2014CA002AE302001710CE0302043E06000000E83F042AE30200171102000000020F01003B
:2014EA0000000F0F9FA002000D1038D80200141058EB0200150F000000303F0400000060F4
:20150A003F04FD2000003E01CE030200220600000000BE5900008000FE5B011108003E01DE
:20152A00000080803E5B2F1F00003E01770302003E0638D802001410000000283F0438D80A
:20154A0002001411FBA002002610F1FFFFFF0C0F20A10200031082EB020002100000000027
:20156A000F0F9FA002006810100000001E0E2FC02C003E019A030204300600000000040F08
:20158A00F09F02003E018A9D020000100D661900040F004011003E01FEFF0000010F0001FB
:2015AA0041003E0104C018003E01000040003E018A9D02000011E1FFFFFF0C0F0CA00D001B
:2015CA003E01030413003E0100000082BE59040000008014C60302003A0608000000801491
:2015EA00C60302003A06003402001F0FF00A0000340F3AD80200440F58EB0200150FF00A6B
:20160A000000360F48CD0200460F38D802001610F00A0000370F3AD80200470F2AE302001E
:20162A00171082EB02000310000000000F0FEAA00200130F9FA002000D100000008EFF71CF
:20164A000000008A7F713FC02C003E01B80302043006882884003E5710A10206BE5D000008
:20166A000022012901000000010D00C85822012900C858003E018C1808003E01000000004F
:20168A00FE5B081008027F5F000000803E5B0000008A7F71000000283F04000000843E59CE
:2016AA00000000F03F04F09F02003E01FD2000003E01AD03020002062AE302001710CE0300
:2016CA0002043E06000000E83F042AE30200171138D80200141058EB0200150F9FA0020074
:2016EA00681000000000BE59030000001E0E00008000FE5B01110800BE59000080803E5B7F
:20170A0001000000200F00000000340F00000000000F001002003E01DC030204000657EBBF
:20172A000200140F0F000000040F01000000000F001002003E01DC030204200602000000EA
:20174A00200F00000000000056EB0200140F56EB0200001160410000010F01007000011162
:20176A0009000000000F009002003E0104000000000D000000003E5804910D003E011100DD
:20178A0010203E0200007000011100000000000F001002003E0135040200000601000000AB
:2017AA00000F001002003E011304020000062DA10200150F00000000350F41EB0200140F17
:2017CA0000000000340F0A000000680F020000001E0E000000003E59000000803E5B57EB1B
:2017EA000200140F02000000260F08000000680F020000001E0E00000000BE59000000803F
:20180A003E5B02800200140F08000000680F020000001E0E000000003E59000000803E5B21
:20182A0055EB02000010000000803E5B57EB02000010000000803E5B56EB02000010000073
:20184A0000803E5BC60000000010FFFCFFFF010F010004003E01C600000000112DA102009B
:20186A00000F30000000001101000000000F3100000000111D000000000F3200000000114D
:20188A00C6000000001000030000010F011004003E01C60000000011350402003E064AA1C0
:2018AA000200150F00000000350F4BEB0200140F00000000340F0A000000680F0200000093
:2018CA001E0E000000003E59000000803E5B58EB0200140F02000000260F08000000680F04
:2018EA00020000001E0E00000000BE59000000803E5B02800200140F08000000680F020058
:20190A0000001E0E000000003E59000000803E5BC60000000010FFFCFFFF010F01000400FD
:20192A003E01C600000000114AA10200000F30000000001101000000000F310000000011F8
:20194A001A000000000F320000000011C6000000001000030000010F011004003E01C6000E
:20196A0000000011350402003E06B80B0000340F4B800200440F038C02001410FCFFFFFFF9
:20198A00260F000000303F04038C0200141140EB0200150F00000000350F948C02002610F2
:2019AA00000000703F0400000000BE5B000000803E5940EB0200150F958C02002610000090
:2019CA0000703F0400000000BE5B000000803E5940EB0200150F968C0200261000000070FF
:2019EA003F0400000000BE5B000000803E5940EB0200150F978C02002610000000703F040B
:201A0A0000000000BE5B000000803E59080000002B14100000002B14200000002B14000493
:201A2A0000002B14000000043E0A800000002B14008002007C101000000080146004020436
:201A4A003A0601000000200FAEA002002110F00A0000300F48CD0200400F640402043E063A
:201A6A0039D802001010FBA002002210F00A0000300F56AC0200400F47B702001010FAA014
:201A8A0002002210A4A002002310B2ED0200001048B70200110F00000000310F00000099E4
:201AAA000F73000000A10F749FA002006810060000001E0E000000890F71000000883E04B8
:201ACA0002000000000D000080003E54000080803E52000000103E04F00A0000300F64A1BB
:201AEA000200400FB2A002000010001002003E017C04020000067EED02001010A4A002007B
:201B0A006810020000001E0E000080003E50000080803E52B3A002000010001002003E01C1
:201B2A008404020000067FED02001010A4A002006810020000001E0E000080003E50000083
:201B4A0080803E52B4A002000010001002003E018C040200000680ED02001010A4A00200C7
:201B6A006810020000001E0E000080003E50000080803E52B5A002000010001002003E015F
:201B8A0000000000000A81ED02001010A4A002006810020000001E0E000080003E500000A7
:201BAA0080803E52000000003E0A48BD0200110F00000000310FF00A0000300F64A102009C
:201BCA00400F01000000200F00000000210FAEA00200221062ED0200120F00000000320F17
:201BEA0000000000330F48BD0200130FABA002000010A3A002000510051500003E01AEA012
:201C0A0002000010502500003E0160ED02000511000080915F70000080801F71000080801F
:201C2A003E54000000583E04000080801F71000080803E54000000583E04000080801F7122
:201C4A00000080803E54000000583E04000080801F71000080803E5448BD0200110FB2A0B3
:201C6A0002000010001002003E01BB04020000067EED02001010000000103E04020000004F
:201C8A00050D000080003E50000080803E52000000D83E04000000803F71000080880F70B9
:201CAA00B3A002000010001002003E01C604020000067FED02001010000000103E040200B0
:201CCA000000050D000080003E50000080803E52000000D83E04000000803F7100008088F8
:201CEA000F70B4A002000010001002003E01D1040200000680ED02001010000000103E04E6
:201D0A0002000000050D000080003E50000080803E52000000D83E04000000803F710000BD
:201D2A0080880F70B5A002000010001002003E01DC040200000681ED0200101000000010D2
:201D4A003E0402000000050D000080003E50000080803E52040000008014000000003A0AA9
:201D6A00ACA002000010A3A002000510051500003E01AEA002000010502500003E0161EDE6
:201D8A0002000511000080915F7066ED0200120F48C50200140F00000000340F0000000056
:201DAA00350FF00A0000300F56AC0200400F47B702001010000000103E04000080980F733D
:201DCA00000080A00F74FAA0020024109FA002006810090000001E0E000080880F71000010
:201DEA0000804F71000000803E540000808A0F7002000000050D000000003E5200000080DA
:201E0A003E5A000000183F04000000203E04000000003E0A01000000000F649502000011FF
:201E2A0003000000000F65950200001153480000000F66950200001141520000000F679523
:201E4A000200001143200000000F68950200001152440000000F69950200001159210000B3
:201E6A00000F6A9502000011200A0000000F6B950200001164950200000F78000000001158
:201E8A0001000000000F79000000001120080000000F7A0000000011879D0200000F68003F
:201EAA000000001101000000000F69000000001101000000000F6A0000000011F364040097
:201ECA00000F859D02000011F0000000001101000F00000FF40000000011F3200400000F69
:201EEA00F10000000011869D02000011002000000D14000800000D14000100000D14010013
:201F0A0000000A14005800000B1400000000000F5F8C02000011618C02000011638C020024
:201F2A000011658C02000011678C02000011698C020000116B8C020000116D8C020000115E
:201F4A006F8C02000011718C02000011A6050200BE06B6050200BE0600010000000F608C6B
:201F6A0002000011628C02000011648C02000011668C02000011688C020000116A8C02003C
:201F8A0000116C8C020000116E8C02000011708C02000011728C02000011A6050200BE067D
:201FAA00B6050200BE0600060000000F06000000010F011004003E01738C02000011758C04
:201FCA0002000011778C02000011798C020000117B8C020000117D8C020000117F8C020073
:201FEA000011818C02000011838C02000011A6050200BE06B6050200BE0600070000000F7C
:20200A0006000000010F011004003E01748C02000011768C02000011788C020000117A8C07
:20202A00020000117C8C020000117E8C02000011808C02000011828C02000011A60502005E
:20204A00BE06B6050200BE06ABC2A245010FBB8C0200011151480000000FA6050200BE0659
:20206A00B6050200BE06B6050200BE0651080000000FA6050200BE06C8000000680F02003A
:20208A0000001E0EB6050200BE0600000000000051070200BE0658140000010F878C0200DA
:2020AA00011100000000020F01420000000F010070000011000070000211888C0200021173
:2020CA0002420000000F010070000011000070000211898C02000211B6050200BE06000AE9
:2020EA000000000FA6050200BE06B6050200BE0609000000000F00A002003E018006000056
:20210A00030F80070000020F8A050200000600A002003E018D050200000600A002003E0118
:20212A0090050200000600A002003E0193050200000600A002003E0196050200000600A053
:20214A0002003E0199050200000600A002003E019C050200000600A002003E019F0502007D
:20216A000006A20502003E0623410000010F01007000011100007000031123410000010F73
:20218A0001007000011100007000021126410000010F01007000011100007000031126414A
:2021AA000000010F01007000011100007000021129410000010F0100700001110000700092
:2021CA00031129410000010F0100700001110000700002112C410000010F01007000011161
:2021EA000000700003112C410000010F010070000111000070000211008F0000000FA60585
:20220A000200BE06B6050200BE06000000003E0A20410000010F01007000011100007000C1
:20222A00001123410000010F01007000011100007000001126410000010F01007000011111
:20224A0000007000001129410000010F0100700001110000700000112C410000010F0100F7
:20226A0070000111000070000011000000003E0AB9050200BE06B9050200BE060000000001
:20228A003E0A0A800200031101000000030F338C02000311338C02000310301302003E010C
:2022AA00BC05020020060A8002000310000000003E0A0C800200140F00000000340F01004F
:2022CA000000240F11800200150F00000000350F868C0200001000A002003E01DD050200DD
:2022EA000206D40502002406FFFFFFFF000F9BEB020000119CEB020000119DEB02000011EE
:20230A00FF000000010FADA002000010011104003E01ADA002000111C08A0000040FD90554
:20232A0002003E0600000000000F9BEB020000119CEB020000119DEB02000011008A0000E6
:20234A00040F05000000680F010000001E0E000000823E5B800602003E06FDFFFFFF040FC3
:20236A00BB8C0200001004910D003E014AED02000010102100003E0100000000240A000032
:20238A000000000F4AED02000011B0ED0200031000000000080FB0ED020008110000000059
:2023AA000F0F130000000C0F04000000020F05000000680F060000001E0E3FC02C003E019A
:2023CA00F20502041006F09F02003E010000000000008C082C003E01C22C00003E010000E4
:2023EA000000090F130000000C0F05000000680F060000001E0E3FC02C003E01FC0502046E
:20240A001006F09F02003E010000000000009C092C003E01C22C00003E019FA0020001103D
:20242A00A1EB02000010012000003E01F2060200A00682EB02000110A2EB020000100120B4
:20244A0000003E01F2060200A0069EEB020003108A8C02000110101102003E010B06020057
:20246A00000611000000070F37032C003E01918C02000110101102003E01100602000006D0
:20248A0010000000070F37032C003E01008A0000040F381304003E0100410000010F0100EA
:2024AA0070000111000070000010000000803E5903410000010F01007000011100007000B2
:2024CA000010000000803E5906410000010F010070000111000070000010000000803E595A
:2024EA0009410000010F010070000111000070000010000000803E590C410000010F010000
:20250A0070000111000070000010000000803E590C800200140FF9EC0200160F00000000DB
:20252A00360F00000000080F00000000070F000000000B0F120000000C0F040000000F0FB6
:20254A0005000000680F260000001E0E000000003E590C000000010F010104003E010400A7
:20256A000000020F122100003E013C06020004063C032C003E0187082C003E0170970200D3
:20258A003E013F0602043E06408A0000040F01000000009D008A0000040F00000000009DAE
:2025AA00709702003E01CF2C00003E014606020024069BEB020003119FEB02000310391390
:2025CA0004003E01120000000C0F010000000B0F30000000010F010104003E0110000000D1
:2025EA00020F122100003E015206020004063C032C003E0180000000010F87082C003E01B6
:20260A00709702003E01540602043E06141404003E0101000000009D00000000009D709717
:20262A0002003E01CF2C00003E01000000823E5BB01B02003E015B06020420069CEB0200D8
:20264A00031101000000000F9BEB02000311001002003E01D80602000006A0EB02000010DC
:20266A00000020008014620602003A06020000000F0F0F002C003E01000000048014680652
:20268A0002043A0682ED02000110101102003E01010000000F0F0F002C003E016D060204F4
:2026AA000006A0EB02000011000000000000040000000F0F0F002C003E010000000180143B
:2026CA00710602003A06030000000F0F0F002C003E01010000008014750602003A06050045
:2026EA0000000F0F0F002C003E010200000080147B0602043A06928C020001100A000000A0
:20270A000C0F060000000F0F0F002C003E011C2100003E017F0602002006070000000F0FA8
:20272A000F002C003E019DEB0200001101000000000F001002003E01D80602000006EC1D2A
:20274A000200BE06B08C020000103E8002000110012100003E01940602002006AA8C02002F
:20276A000010418002000110012100003E01940602002006AB8C020002104080020001102A
:20278A00212100003E01940602002006AF8C020002103F8002000110212200003E01D8066B
:2027AA0002000006B08C020002103E8002000211AF8C020002103F8002000211AB8C020088
:2027CA000210408002000211AA8C02000210418002000211AA8C02000010001002003E014F
:2027EA00D8060200000602000000010F012100003E01B406020020060A000000000F928C5D
:20280A0002000011B08C0200001002000000010F012100003E01AB0602002006C506020430
:20282A003E0602000000001401000000001403000000010F012100003E01B10602002006CC
:20284A00C50602043E06020000002014010000000014C50602043E060200000000140100E2
:20286A0000002014AB8C0200001003000000010F102100003E01BB06020020060100000064
:20288A00000F928C02000011C50602003E0602000000010F102100003E01C306020020066A
:2028AA000A000000000F928C02000011C50602043E06020000002014010000002014000044
:2028CA000000000F928C02000011AF8C0200001000000000010F012100003E01CE0602001A
:2028EA00200601000000000F8A8C02000011D70602043E0600000000000F918C0200001109
:20290A0000000000010F8A8C0200011103000000010F012100003E01D70602040006010015
:20292A000000000F918C0200001101000000000F8A8C020000110000000000001180020082
:20294A00150F20410000010F010070000111000000003E5B00007000001123410000010FC7
:20296A00010070000111000000003E5B00007000001126410000010F0100700001110000B6
:20298A0000003E5B00007000001129410000010F010070000111000000003E5B000070000D
:2029AA0000112C410000010F010070000111000000003E5B000070000011ADA00200001083
:2029CA00081004003E01ADA002000011B6050200BE06000000003E0A00000000000F9FA01B
:2029EA0002000110A1EB02000111101102003E0107070200000610A102003E01070702049C
:202A0A0000060D000000070F07002C003E0110A102003E0107070204000609000000070FE6
:202A2A0007002C003E0110A102003E0107070204000605000000070F07002C003E0110A1D0
:202A4A0002003E0107070204000601000000070F07002C003E0182EB02000310A2EB020077
:202A6A000311000000000F0F3FC02C003E010E07020030060C000000070F07002C003E01CF
:202A8A00F09F02003E013FC02C003E0113070200300608000000070F07002C003E01F09F81
:202AAA0002003E013FC02C003E0118070200300604000000070F07002C003E01F09F0200ED
:202ACA003E013FC02C003E011D070200300600000000070F07002C003E01F09F02003E018F
:202AEA009EEB0200001100000000000F9FA00200011004000000070F172100003E015007E7
:202B0A000200040610A102003E0138070204000611000000070F07002C003E0110A1020016
:202B2A003E013807020400060D000000070F07002C003E0110A102003E013807020400062F
:202B4A0009000000070F07002C003E0110A102003E0138070204000605000000070F07007B
:202B6A002C003E0110A102003E0138070204000601000000070F07002C003E013FC02C00EF
:202B8A003E013C070200300610000000070F07002C003E01F09F02003E013FC02C003E019F
:202BAA004107020030060C000000070F07002C003E01F09F02003E013FC02C003E01460770
:202BCA000200300608000000070F07002C003E01F09F02003E013FC02C003E014B07020095
:202BEA00300604000000070F07002C003E01F09F02003E013FC02C003E0150070200300640
:202C0A0000000000070F07002C003E019FEB02000011BB8C02000010B48C02000C107F0748
:202C2A000200BE06000000860F70DB0FC940000F7F070200BE062C8C0200001100000000A6
:202C4A00070F2F8C020007118E8C02000710701702003E016C07020000062C8C020000103F
:202C6A00000000000C0F308C02000C118F8C02006810010000001E0E0C1C08003E012D8C6A
:202C8A0002000C112C8C02000010000000000C0F318C02000C11908C0200681001000000B3
:202CAA001E0E0C1C08003E012E8C02000C11000000003E0ABB8C02000010B58C02000C1096
:202CCA007F070200BE06000000860F70DB0FC940000F7F070200BE062D8C0200001100007F
:202CEA000000070F318C02000711BB8C02000010B68C02000C107F070200BE060000008652
:202D0A000F70DB0FC940000F7F070200BE062D8C0200001100000000070F318C0200071123
:202D2A00000000003E0A000000400B0FC0408C830F700C0C13003E013C7059003E010C0C93
:202D4A0013003E013C7059003E010C0C13043E0A3C7059003E01070013003E0142800200FB
:202D6A0000114380020001114480020002114580020010114680020020114780020030119D
:202D8A00488002007C1100000000300F879D02000010000010103E02889D020001101011A4
:202DAA0000003E0111F802783E02889D020001114A800200011000FFFFFF020F12010400CC
:202DCA003E01101100003E010A0A0A0A020F122200003E01AF0702000006110802003E0285
:202DEA004A8002000111899D02000010009002003E01899D02000011108010003E02C20700
:202E0A000200300610FE01783E0210A102003E01000000901F70448D0200100F889D02007F
:202E2A000110000080803E4000000000010F889D0200011110040000010F01A000003E01AC
:202E4A00C20702000206899D02000010108010003E02B70702001006009002003E01889DB1
:202E6A000200011011F802783E02889D02000111B00702003E06899D0200001010FE01787D
:202E8A003E02000000901F70448D0200100F889D02000110000080803E4000000000000F12
:202EAA00899D02000011889D0200001101000000000F849D02000011879D0200000F6800B6
:202ECA000000001101000000000F69000000001101000000000F6A000000001100000000C2
:202EEA00000FF10000000011869D02000010F100000000114780020030104680020020107F
:202F0A00458002001010448002000210438002000110000000043E0A42800200001048802A
:202F2A0002007C10000000003E0A00000000011000700000020F121104003E0100000000B9
:202F4A00011102000000011000FCFFFF020F120104003E0121020000020F121104003E0147
:202F6A00020000000111348C0200100F01000000200F00000000300F80000000680F0100EB
:202F8A0000001E0E00000000009001000000000FB4ED02000011B48C0200100F0100000045
:202FAA00200F00000000300F10000000680F010000001E0E00000000009002000000000F44
:202FCA00B4ED020000110A000000000F368C0200001105420000010F01007000011100006B
:202FEA007000001109000000000F378C0200001106420000010F01007000011100900200EB
:20300A003E0100007000001100000000000F928C0200001100000000000F868C0200001172
:20302A0058140000000F878C02000011ABC2A245010FBB8C0200011100000000000F888C03
:20304A0002000011898C020000111E000000000FAEA00200001104000000000F938C020069
:20306A00001117000000000F948C0200001117000000000F958C0200001117000000000F5C
:20308A00968C0200001117000000000F978C02000011FF3F0000000F00000000010F0E9E8C
:2030AA00020000110F9E02000111109E02000111119E02000111129E02000111139E020036
:2030CA000011149E02000111159E02000111169E02000111179E0200011102000000000FA6
:2030EA0001430000010F01007000011114000000680F010000001E0E00007000001115435E
:20310A000000010F01007000011111000000680F010000001E0E00007000001100000000DC
:20312A00340F01000000240F00000000010F00010000000F1B0B0200BE0620010000000FD2
:20314A001B0B0200BE0640010000000F1B0B0200BE0660010000000F1B0B0200BE06800160
:20316A000000000F1B0B0200BE06A0010000000F1B0B0200BE06C0010000000F1B0B0200B6
:20318A00BE06E0010000000F1B0B0200BE0600020000000F1B0B0200BE0620020000000F57
:2031AA001B0B0200BE0640020000000F1B0B0200BE0660020000000F1B0B0200BE068002FD
:2031CA000000000F1B0B0200BE06A0020000000F1B0B0200BE06C0020000000F1B0B020054
:2031EA00BE06E0020000000F1B0B0200BE0600030000000F1B0B0200BE0620030000000FF4
:20320A001B0B0200BE0640030000000F1B0B0200BE0660030000000F1B0B0200BE06800399
:20322A000000000F1B0B0200BE06A0030000000F1B0B0200BE06C0030000000F1B0B0200F1
:20324A00BE06E0030000000F1B0B0200BE0600040000000F1B0B0200BE0620040000000F90
:20326A001B0B0200BE0640040000000F1B0B0200BE0660040000000F1B0B0200BE06800436
:20328A000000000F1B0B0200BE06A0040000000F1B0B0200BE06C0040000000F1B0B02008F
:2032AA00BE06E0040000000F1B0B0200BE0600050000000F1B0B0200BE0620050000000F2D
:2032CA001B0B0200BE0640050000000F1B0B0200BE0660050000000F1B0B0200BE068005D3
:2032EA000000000F1B0B0200BE0603420000000F01007000001101000000010F0000700072
:20330A00011104420000000F010070000011000070000111848C02000111858C02000111EF
:20332A000A420000000F01007000001101000000020F14000000680F010000001E0E0000DC
:20334A00700002111E420000000F01007000001101000000020F11000000680F0100000054
:20336A001E0E00007000021100000100000F3A8C0200140F00000000340F01000000240F22
:20338A0014000000680F010000001E0E000000803E594E8C0200140F11000000680F0100CC
:2033AA0000001E0E000000803E5901000000000F8A8C0200001101000000000F8B8C02005E
:2033CA00001100000000000F8C8C0200001100000000000F8D8C0200001100000000000F4E
:2033EA00918C0200001101000000000F8E8C0200001102000000000F8F8C02000011030014
:20340A000000000F908C020000110000C842000FB48C0200001100004843000FB58C02001B
:20342A00001100009643000FB68C020000110000003F000FB78C02000011CDCC4C3E000F5E
:20344A00B88C02000011CDCC4C3E000FB98C020000110000003F000FBA8C020000118E9DAF
:20346A000200140FCE9D0200150F00000000350F2D9E020000993C9E020000100000008076
:20348A003E5B3D9E020000994C9E02000010000000803E5B4D9E020000995C9E020000106C
:2034AA00000000803E5B5D9E020000996C9E02000010000000803E5B6D9E020000997C9E5E
:2034CA0002000010000000803E5B7D9E020000998C9E02000010000000803E5B8D9E02007F
:2034EA0000999C9E02000010000000803E5B9D9E02000099AC9E02000010000000803E5B79
:20350A00AD9E02000099BC9E02000010000000803E5BBD9E02000099CC9E020000100000C4
:20352A0000803E5BCD9E02000099DC9E02000010000000803E5BDD9E02000099EC9E02001B
:20354A000010000000803E5BED9E02000099FC9E02000010000000803E5BFD9E0200009917
:20356A000C9F02000010000000803E5B0D9F020000991C9F02000010000000803E5B1D9F82
:20358A00020000992C9F02000010000000803E5B2D9F020000993C9F0200001000000080BC
:2035AA003E5B3D9F020000994C9F02000010000000803E5B4D9F020000995C9F0200001047
:2035CA00000000803E5B5D9F020000996C9F02000010000000803E5B6D9F020000997C9F39
:2035EA0002000010000000803E5B7D9F020000998C9F02000010000000803E5B8D9F02005B
:20360A0000999C9F02000010000000803E5B9D9F02000099AC9F02000010000000803E5B54
:20362A00AD9F02000099BC9F02000010000000803E5BBD9F02000099CC9F0200001000009F
:20364A0000803E5BCD9F02000099DC9F02000010000000803E5BDD9F02000099EC9F0200F6
:20366A000010000000803E5BED9F02000099FC9F02000010000000803E5BFD9F02000099F3
:20368A000CA002000010000000803E5B0DA0020000991CA002000010000000803E5B1DA05D
:2036AA00020000992CA002000010000000803E5B2DA0020000993CA0020000100000008098
:2036CA003E5B3DA0020000994CA002000010000000803E5B4DA0020000995CA00200001022
:2036EA00000000803E5B5DA0020000996CA002000010000000803E5B6DA0020000997CA014
:20370A0002000010000000803E5B7DA0020000998CA002000010000000803E5B8DA0020036
:20372A0000999CA002000010000000803E5B0100000000140200000000140400000020141C
:20374A00080000000014100000000014200000000014400000000014800000002014AAA099
:20376A000200701101000000000FB6A00200001102000000000FB7A00200001104000000C4
:20378A00000FB8A00200001108000000000FB9A00200001110000000000FBAA00200001196
:2037AA0020000000000FBBA00200001140000000000FBCA00200001180000000000FBDA0B8
:2037CA000200001100010000000FBEA00200001100020000000FBFA00200001100040000C4
:2037EA00000FC0A00200001100080000000FC1A00200001100100000000FC2A0020000111E
:20380A0000200000000FC3A00200001100400000000FC4A00200001100800000000FC5A03F
:20382A000200001100000000000FC6A002000011C7A002000011C8A002000011C9A0020083
:20384A00001101000000000FCAA002000011CBA002000011CCA002000011CDA00200001143
:20386A00CEA002000011CFA002000011D0A002000011D1A002000011D2A002000011D3A03C
:20388A0002000011D4A002000011D5A002000011D6A002000011D7A002000011D8A002006F
:2038AA000011D9A00200001120000000000FABA002000011DAA002000011DBA002000011B9
:2038CA00DCA002000011DDA002000011DEA002000011DFA002000011E0A002000011E1A088
:2038EA0002000011E2A002000011E3A002000011E4A002000011E5A002000011E6A00200C9
:20390A000011E7A002000011E8A002000011E9A002000011ACA002000011EAA002000011BF
:20392A00EBA002000011ECA002000011EDA002000011EEA002000011EFA002000011F0A0CD
:20394A0002000011F1A002000011F2A002000011F3A002000011F4A002000011F5A002001D
:20396A000011F6A002000011F7A002000011F8A002000011F9A00200001140000000000F33
:20398A00A3A00200001120000000000FA4A002000011A3A002000010AEA002000110012268
:2039AA0000003E01B2ED0200021120A202003E01B1ED02000211A4A00200001000A002005C
:2039CA003E01B3ED0200001101000000000F9EA002000011F00A0000000FFCA002000011D2
:2039EA0001000000000FB2A00200001100000000000FB3A002000011B4A002000011B5A017
:203A0A000200001101000000000F9FA002000011FEFFFFFF000FA9A00200001100000000C1
:203A2A00000F001002003E01B0090200000601000000000F001002003E01B0090200200619
:203A4A00FFFFFFFF000FA9A00200001100040000000FFEA002000011FDA002000011F00A87
:203A6A000000000FFAA002000011F00A0000000FFBA00200001101000000000FA0A0020077
:203A8A0000110000803E000F1FA102000011CDCCCC3D000F20A1020000110AD7233C000F97
:203AAA001DA1020000116F12833A010F1EA102000111010013003E010000803F010F1021B7
:203ACA0008003E0183EB020001110DED0200100F00000000300F01000000200F1400000075
:203AEA00680F010000001E0E000080803E50D8E60200100FBC000000680F010000001E0E4B
:203B0A0000000000009001000000000FD8E60200001115000000000FD9E602000011000034
:203B2A00803F000FDAE6020000112CE30200100F00000000300F01000000200FAC0300008C
:203B4A00680F010000001E0E0000000000902CE30200100F02000000000F0000803F010F17
:203B6A0010000000680F040000001E0E010000000090000000803E50000080803E500090C7
:203B8A0002003E01F9EC0200100F14000000680F010000001E0E000000000090B80B0000C9
:203BAA00340F4B800200440F038C0200141101000000240FB80B0000680F010000001E0E47
:203BCA00000000000099000001002014000002002014000004002014000008000014000083
:203BEA001000001400000000000FADA00200001105000000000FA6A002000011A5A0020074
:203C0A0000110B100000000F358C0200001104000000000FAC8C0200001109000000000F15
:203C2A00AD8C020000110A000000000FAE8C020000110A000000000F368C020000110900D1
:203C4A000000000F378C0200001166000000000FB38C0200001100000080AF77000000C048
:203C6A00010F010104003E0111E200783E02B18C0200011100000030010F010104003E0164
:203C8A0011E400783E02B28C0200011101000000010FA98C0200011100002000201400006D
:203CAA0040002014000080002014000000012014000000022014000000042014000000002F
:203CCA00000F80EB0200001181EB02000011F7EC02000011F8EC0200001149ED0200001198
:203CEA0082ED020000114BED020000119BED02000011A7A002000011A8A00200001184ED2C
:203D0A000200001186ED02000011A0EB020000114AED020000119FA002000110A1EB020038
:203D2A000111101102003E013B0A0200000610A102003E013B0A020400060D000000070F52
:203D4A0007002C003E0110A102003E013B0A0204000609000000070F07002C003E0110A162
:203D6A0002003E013B0A0204000605000000070F07002C003E0110A102003E013B0A0204DD
:203D8A00000601000000070F07002C003E0182EB02000310A2EB02000311000000000F0F47
:203DAA003FC02C003E01420A020030060C000000070F07002C003E01F09F02003E013FC0A8
:203DCA002C003E01470A0200300608000000070F07002C003E01F09F02003E013FC02C005A
:203DEA003E014C0A0200300604000000070F07002C003E01F09F02003E013FC02C003E0126
:203E0A00510A0200300600000000070F07002C003E01F09F02003E019EEB02000011000011
:203E2A000000000F9FA00200011004000000070F172100003E01840A0200040610A1020039
:203E4A003E016C0A0204000611000000070F07002C003E0110A102003E016C0A020400068A
:203E6A000D000000070F07002C003E0110A102003E016C0A0204000609000000070F070009
:203E8A002C003E0110A102003E016C0A0204000605000000070F07002C003E0110A10200F9
:203EAA003E016C0A0204000601000000070F07002C003E013FC02C003E01700A0200300692
:203ECA0010000000070F07002C003E01F09F02003E013FC02C003E01750A020030060C0043
:203EEA000000070F07002C003E01F09F02003E013FC02C003E017A0A020030060800000032
:203F0A00070F07002C003E01F09F02003E013FC02C003E017F0A0200300604000000070FFA
:203F2A0007002C003E01F09F02003E013FC02C003E01840A0200300600000000070F0700E8
:203F4A002C003E019FEB02000011A9A00200011082EB020001111DA1020000101EA10200E1
:203F6A000110010013003E010000803F010F102108003E0183EB020001110DED0200100FEF
:203F8A0000000000300F01000000200F14000000680F010000001E0E000080803E50F00A68
:203FAA000000300F64A10200400F54AC02001011F00A0000680F010000001E0E00000000A1
:203FCA000090F00A0000300F56AC0200400F46B702001011F00A0000680F010000001E0EFD
:203FEA0000000000009000A00000300F00604200400F000043001011F00A0000680F010081
:20400A0000001E0E00000000009000A00000300F02004300400F02A043001011F00A000067
:20402A00680F010000001E0E000000000090F00A0000300F3AD80200400F2AE30200101176
:20404A00F00A0000680F010000001E0E000000000090F00A0000300F48CD0200400F38D879
:20406A0002001011F00A0000680F010000001E0E00000000009040EB0200140F0000000095
:20408A00340F01000000240F40000000680F010000001E0E00000000009921ED0200100FF3
:2040AA0000000000300F01000000200F14000000680F010000001E0E0000000000904CED06
:2040CA000200100F6F12833A000F14000000680F010000001E0E000000803E5035ED02007E
:2040EA00100F14000000680F010000001E0E0000000000901DA102000010A3EB0200100FD0
:20410A00A0000000680F010000001E0E000000803E501DA1020000100000803E010F0100A4
:20412A0013003E0143EC0200100FA0000000680F010000001E0E000000803E50003002004F
:20414A00180F00000000380F01000000280F00000000080F99EB02000010001002003E01B1
:20416A00E90A0200000600040000680F010000001E0E000000843F5000340200180F000022
:20418A000000380F01000000280F00000000080F00040000680F010000001E0E0000008453
:2041AA003F5001000000000F99EB0200001100000000380F00004200180F01000000280FD7
:2041CA0017B7D138080F9AEB02000010001002003E010E0B0200000600600000680F010006
:2041EA0000001E0E000000843F5000004200180F00004200190F00000000390FFDA00200BC
:20420A002910800000002A0F00000000000F00000000040FA0A0020005109FA002000210D6
:20422A0000000000010FAEA002006810010000001E0E000000803F50000000487E04000096
:20424A00008C9F71109102003E01122300003E01FF0A02000206000000507E04000000502D
:20426A007E04000000507E04000000507E04409402003E01452600003E01FE0A020002063D
:20428A0001000000000F9AEB0200001155380200180F00000000000F00060000680F010029
:2042AA0000001E0E000000803F50553E0200180F00000000000F00060000680F0100000070
:2042CA001E0E000000803F50000000003E0A0E9E0200140F0100700000110A000000680F7D
:2042EA00030000001E0E000000003E59000070000011000070000111000000003E0A448DD2
:20430A00020002100000FFFF010F210204003E0122F002783E0243310000010F1221000088
:20432A003E012C0B0200000641430000010FCE1502002006458D02000110BFED02000111B1
:20434A00FF000000020F120204003E0147000000030F232200003E01FC1002002206414454
:20436A005021020F212200003E01430B02002006468D02000110101102003E013B0B020029
:20438A0000060100000000143C0B02003E06010000002014478D02000110101102003E01ED
:2043AA00410B02000006020000000014420B02003E06020000002014D81502003E06414C00
:2043CA004721020F212200003E01650B02002006468D020001101DA102000111478D0200B2
:2043EA000110101102003E014D0B020000064000000000144E0B02003E0640000000201479
:20440A00488D020001101EA102000111498D02000110101102003E01550B02000006200004
:20442A0000000014560B02003E062000000020144A8D02000110A5A0020001114B8D020046
:20444A000110101102003E015D0B020000062000000000145E0B02003E06800000002014D8
:20446A001DA1020000101EA102000110010013003E010000803F010F102108003E0183EB88
:20448A0002000111D81502003E0641534421020F212200003E016F0B02002006468D0200C8
:2044AA000110A9A00200011182EB02000210D81502043E06121204003E0182EB02000211E3
:2044CA00D81502003E0642415544020F212200003E018A0B02002006468D020001108025A8
:2044EA000000020F122200003E01780B02002006BB200000000F860B02003E06004B000077
:20450A00020F122200003E017D0B02002006CC200000000F860B02003E0600E10000020F99
:20452A00122200003E01820B0200200688200000000F860B02003E0600C20100020F1222B3
:20454A0000003E01760B0200200666200000000F00420000010F010070000111000070008F
:20456A000011CE1502003E0643415421020F212200003E012A0C02002006468D0200011027
:20458A00478D0200021010A102003E01980B02002006738C02000110C0FFFFFF000F01018C
:2045AA0004003E01121104003E01738C0200011120410000000F260C02003E0610A102009A
:2045CA003E01A10B02002006748C02000110C0FFFFFF000F010104003E01121104003E0134
:2045EA00748C0200011120410000000F260C02003E0610A102003E01AA0B02002006758CE5
:20460A0002000110C0FFFFFF000F010104003E01121104003E01758C02000111234100008D
:20462A00000F260C02003E0610A102003E01B30B02002006768C02000110C0FFFFFF000F30
:20464A00010104003E01121104003E01768C0200011123410000000F260C02003E0610A1F3
:20466A0002003E01BC0B02002006778C02000110C0FFFFFF000F010104003E0112110400B2
:20468A003E01778C0200011126410000000F260C02003E0610A102003E01C50B02002006E2
:2046AA00788C02000110C0FFFFFF000F010104003E01121104003E01788C020001112641E3
:2046CA000000000F260C02003E0610A102003E01CE0B02002006798C02000110C0FFFFFF81
:2046EA00000F010104003E01121104003E01798C0200011129410000000F260C02003E06EC
:20470A0010A102003E01D70B020020067A8C02000110C0FFFFFF000F010104003E01121146
:20472A0004003E017A8C0200011129410000000F260C02003E0610A102003E01E00B020042
:20474A0020067B8C02000110C0FFFFFF000F010104003E01121104003E017B8C020001117D
:20476A002C410000000F260C02003E0610A102003E01E90B020020067C8C02000110C0FF53
:20478A00FFFF000F010104003E01121104003E017C8C020001112C410000000F260C02008B
:2047AA003E0610A102003E01F20B020020067D8C02000110C0FFFFFF000F010104003E0167
:2047CA00121104003E017D8C020001112F410000000F260C02003E0610A102003E01FB0B5D
:2047EA00020020067E8C02000110C0FFFFFF000F010104003E01121104003E017E8C0200E7
:20480A0001112F410000000F260C02003E0610A102003E01040C020020067F8C020001103D
:20482A00C0FFFFFF000F010104003E01121104003E017F8C0200011132410000000F260C24
:20484A0002003E0610A102003E010D0C02002006808C02000110C0FFFFFF000F01010400E4
:20486A003E01121104003E01808C0200011132410000000F260C02003E0610A102003E017D
:20488A00160C02002006818C02000110C0FFFFFF000F010104003E01121104003E01818C20
:2048AA000200011135410000000F260C02003E0610A102003E011F0C02002006828C020088
:2048CA000110C0FFFFFF000F010104003E01121104003E01828C0200011135410000000F9F
:2048EA00260C02003E06838C02000110C0FFFFFF000F010104003E01121104003E01838C8E
:20490A000200011138410000000F260C02003E06010070000011000070000111B6050200B8
:20492A00BE06D81502003E0643414C3F020F212200003E013F0C0200200601000000240F2D
:20494A0000000000340F1DA10200140F64950200110F00000000310F04000000210F000098
:20496A0000483E0401000000210F10000000080F809002003E0165950200001104000000E9
:20498A00080D000080007E58000080807E5211F000783E02000080807E52D1150200BE069D
:2049AA00C21502003E0643414E21020F212200003E015D0C02002006468D0200110F0000C4
:2049CA000000310F01000000210F9DA00200140F00000000340F80000000680F02000000BE
:2049EA001E0E000000007E52000000807E581DA10200140F00000000340F10000000680FAE
:204A0A00020000001E0E000000007E52000000807E5814170200BE0601000000010F328C78
:204A2A000200011100430000000F01007000001100007000011100100000010F00420000A0
:204A4A00000F010070000011000070000111F9090200BE06D81502003E064341583F020F12
:204A6A00212200003E01730C02002006AAA00200701101000000240F00000000340F9DA082
:204A8A000200140F64950200110F00000000310F04000000210F000000483E0401000000CD
:204AAA00210F80000000080F809002003E0165950200001104000000080D000080007E5858
:204ACA00000080807E5211F000783E02000080807E52D1150200BE06C21502003E06434225
:204AEA004C3F020F212200003E01880C0200200601000000240F00000000340FB48C020019
:204B0A00140F64950200110F00000000310F04000000210F000000483E0401000000210F1E
:204B2A0010000000080F809002003E0165950200001104000000080D000080007E58000077
:204B4A0080807E5211F000783E02000080807E52D1150200BE06C21502003E064342583F0D
:204B6A00020F212200003E019D0C0200200601000000240F00000000340F348C0200140F6B
:204B8A0064950200110F00000000310F04000000210F000000483E0401000000210F800041
:204BAA000000080F809002003E0165950200001104000000080D000080007E580000808007
:204BCA007E5211F000783E02000080807E52D1150200BE06C21502003E0643424E21020FA4
:204BEA00212200003E01B50C0200200600430000000F01007000001100000000000F00005D
:204C0A0070000011328C02000011468D0200110F00000000310F01000000210FC48C020080
:204C2A00140F00000000340F80000000680F020000001E0E000000007E52000000807E58B9
:204C4A00B48C0200140F00000000340F10000000680F020000001E0E000000007E5200001D
:204C6A0000807E58D81502003E0643474E21020F212200003E01700D02002006468D02009B
:204C8A000110478D0200021010A102003E01C30C020020065F8C02000110F0FFFFFF000F2E
:204CAA00010104003E01121104003E015F8C0200011120410000000F6C0D02003E0610A160
:204CCA0002003E01CC0C02002006608C02000110F0FFFFFF000F010104003E011211040022
:204CEA003E01608C0200011120410000000F6C0D02003E0610A102003E01D50C0200200641
:204D0A00618C02000110F0FFFFFF000F010104003E01121104003E01618C0200011123417D
:204D2A000000000F6C0D02003E0610A102003E01DE0C02002006628C02000110F0FFFFFFA9
:204D4A00000F010104003E01121104003E01628C0200011123410000000F6C0D02003E065B
:204D6A0010A102003E01E70C02002006638C02000110F0FFFFFF000F010104003E011211B6
:204D8A0004003E01638C0200011126410000000F6C0D02003E0610A102003E01F00C02009E
:204DAA002006648C02000110F0FFFFFF000F010104003E01121104003E01648C0200011115
:204DCA0026410000000F6C0D02003E0610A102003E01F90C02002006658C02000110F0FF82
:204DEA00FFFF000F010104003E01121104003E01658C0200011129410000000F6C0D0200F8
:204E0A003E0610A102003E01020D02002006668C02000110F0FFFFFF000F010104003E01D5
:204E2A00121104003E01668C0200011129410000000F6C0D02003E0610A102003E010B0DBA
:204E4A0002002006678C02000110F0FFFFFF000F010104003E01121104003E01678C02007E
:204E6A0001112C410000000F6C0D02003E0610A102003E01140D02002006688C0200011099
:204E8A00F0FFFFFF000F010104003E01121104003E01688C020001112C410000000F6C0D64
:204EAA0002003E0610A102003E011D0D02002006698C02000110F0FFFFFF000F0101040054
:204ECA003E01121104003E01698C020001112F410000000F6C0D02003E0610A102003E01EA
:204EEA00260D020020066A8C02000110F0FFFFFF000F010104003E01121104003E016A8CA7
:204F0A00020001112F410000000F6C0D02003E0610A102003E012F0D020020066B8C0200E6
:204F2A000110F0FFFFFF000F010104003E01121104003E016B8C0200011132410000000F22
:204F4A006C0D02003E0610A102003E01380D020020066C8C02000110F0FFFFFF000F010120
:204F6A0004003E01121104003E016C8C0200011132410000000F6C0D02003E0610A102007E
:204F8A003E01410D020020066D8C02000110F0FFFFFF000F010104003E01121104003E019F
:204FAA006D8C0200011135410000000F6C0D02003E0610A102003E014A0D020020066E8C2B
:204FCA0002000110F0FFFFFF000F010104003E01121104003E016E8C020001113541000089
:204FEA00000F6C0D02003E0610A102003E01530D020020066F8C02000110F0FFFFFF000F55
:20500A00010104003E01121104003E016F8C0200011138410000000F6C0D02003E0610A1D4
:20502A0002003E015C0D02002006708C02000110F0FFFFFF000F010104003E01121104001D
:20504A003E01708C0200011138410000000F6C0D02003E0610A102003E01650D0200200624
:20506A00718C02000110F0FFFFFF000F010104003E01121104003E01718C020001113B41E2
:20508A000000000F6C0D02003E06728C02000110F0FFFFFF000F010104003E0112110400BF
:2050AA003E01728C020001113B410000000F6C0D02003E0601007000001100007000011147
:2050CA00B6050200BE06D81502003E06434E5221020F212200003E01E00D02002006004323
:2050EA000000000F01007000001100000000000F000070000011328C020000110042000072
:20510A00000F01007000001100100000000F00007000001100000000000F99EB02000011AE
:20512A009AEB02000011F9090200BE0601000000240F00000000340F00005000150F00001A
:20514A000000350F00000000380F01000000280F000000003E5B000010103E02A5000000E4
:20516A00030F032000003E01B40D02002006C48C0200140F80000000680FBC0D0200BE06CD
:20518A00B48C0200140F10000000680FBC0D0200BE069DA00200140F80000000680FBC0D68
:2051AA000200BE061DA10200140F10000000680FBC0D0200BE0600004200180F006000005D
:2051CA00680FCE0D0200BE0600300200180F00040000680FCE0D0200BE0600340200180FDB
:2051EA0000040000680FCE0D0200BE06D8E60200140FBC000000680FBC0D0200BE062CE3D5
:20520A000200140FAC030000680FBC0D0200BE0600000000000F99EB020000119AEB02007D
:20522A00001114170200BE0601000000010F328C0200011100430000000F010070000011AB
:20524A0000007000011100100000010F00420000000F010070000011000070000111D81560
:20526A0002003E0601000000010F328C0200011100430000000F01007000001100007000B7
:20528A000111434E5621010FBFED02000111D81502003E06100000001E0E000000003E5B12
:2052AA00000010103E0210F802783E02000000003E5B000010103E02101100003E0111F860
:2052CA0002783E02000000003E5B000010103E02101100003E0111F802783E0200000000EE
:2052EA003E5B000010103E02101100003E0111F802783E02000080803E59000000003E0AA9
:20530A00100000001E0E000000003E5B000010103E0210F802783E02000000003E5B0000F3
:20532A0010103E02101100003E0111F802783E02000000003E5B000010103E0210110000C6
:20534A003E0111F802783E02000000003E5B000010103E02101100003E0111F802783E0225
:20536A00000080803F50000000003E0A434E5321020F212200003E014B0E02002006AA0089
:20538A000000000F55000000010F80000000020F10000000030F555550000011AA2A5000AD
:2053AA000111555550000211555550000011AA2A500001115555500003110A00000000006B
:2053CA000300ED0D02000E00000000003900F00D0200000050000B10000050000C10BC2BC0
:2053EA0000003E01F00D0200200601000000240F00000000340F00005000150F0000000054
:20540A00350F00000000250FAA000000000F55000000010FA0000000020FA5000000030F84
:20542A003F0E0200BE06000000603F04348C0200140F80000000680F1D0E0200BE06B48C9F
:20544A000200140F10000000680F1D0E0200BE069DA00200140F80000000680F1D0E02001F
:20546A00BE061DA10200140F10000000680F1D0E0200BE0600000000380F00004200180F53
:20548A0001000000280F00600000680F2E0E0200BE0600300200180F00040000680F2E0EE1
:2054AA000200BE0600340200180F00040000680F2E0E0200BE06D8E60200140FBC000000A3
:2054CA00680F1D0E0200BE062CE30200140FAC030000680F1D0E0200BE06D81502003E06DC
:2054EA000F0000001E0E000080013E593F0E0200BE06000000603F0433F800783E023F0E69
:20550A000200BE06000000603F0433F800783E023F0E0200BE06000000603F0433F80078DC
:20552A003E023F0E0200BE060A00000000000300290E02000E00000000000E002C0E020070
:20554A00000000603F04000000003E0A0F0000001E0E000080013F503F0E0200BE060000F8
:20556A0000603F0433F800783E023F0E0200BE06000000603F0433F800783E023F0E0200B3
:20558A00BE06000000603F0433F800783E023F0E0200BE060A000000000003003A0E02004D
:2055AA000E0000000000B00F3D0E0200000000603F04000000003E0A555550000011AA2AFD
:2055CA0050000111555550000211000080817E5B0000000000000000000000000000000276
:2055EA007E5B000000000000000080027E5B452400003E01450E02002006000000003E0A02
:20560A0044415421020F212200003E018E0E0200200601020000000F659502000011468D3D
:20562A0002000210938C0200021120A102003E01560E0200200600020000030F5B0E02000B
:20564A003E0610A102003E015A0E0200200600010000030F5B0E02003E0680000000030F26
:20566A00478D02000410488D02000510498D020006104A8D02000710B80B0000340F4B809B
:20568A000200440F04000000240F64950200110F00000000310F000000603E040100000076
:2056AA00210F401402003E016E0E02000006038C0200141004000000030D000080003E59B7
:2056CA00000080807E5211F000783E02000080807E52501502003E01770E02000006038CA5
:2056EA0002001410000000083F0404000000030D000080003E59000080807E5211F00078BB
:20570A003E02000080807E52601602003E01810E02000006038C02001410000000083F0421
:20572A00000000083F0404000000030D000080003E59000080807E5211F000783E02000060
:20574A0080807E52701702003E018C0E02000006038C02001410000000083F0400000008FD
:20576A003F04000000083F0404000000030D000080003E59000080807E5211F000783E02DD
:20578A00000080807E52D1150200BE06C21502003E0644535221020F212200003E01A20E19
:2057AA0002002006468D02000110478D0200021010A102003E01000000921F7000000000D6
:2057CA00340F948C0200140F000000203F04000000813E59B80B0000340F4B800200440F96
:2057EA00038C02001410000000203F0404000000240F00020000680F010000001E0E0000AA
:20580A0000000099D81502003E0645424321020F212200003E01CE0E02002006468D02005B
:20582A000010B6A002000011478D02000010B7A002000011488D02000010B8A00200001143
:20584A00498D02000010B9A0020000114A8D02000010BAA0020000114B8D02000010BBA04F
:20586A00020000114C8D02000010BCA0020000114D8D02000010BDA0020000114E8D020078
:20588A000010BEA0020000114F8D02000010BFA002000011508D02000010C0A002000011BB
:2058AA00518D02000010C1A002000011528D02000010C2A002000011538D02000010C3A0BF
:2058CA0002000011548D02000010C4A002000011558D02000010C5A002000011568D0200F0
:2058EA000010C6A002000011578D02000010C7A002000011588D02000010C8A00200001133
:20590A00D81502043E06598D02000010C9A00200001146454E21020F212200003E01DC0E5B
:20592A0002002006468D0200011003420000000F010070000011000070000111848C0200E5
:20594A000111478D0200011004420000000F010070000011000070000111858C02000111C6
:20596A00D81502003E06464C5421020F212200003E01BD100200200600000000010F328C8D
:20598A000200011100430000000F010070000011000070000111468D02000110101102008A
:2059AA003E01DE0F02002006478D02000010488D02000210001102003E01800F02000006D1
:2059CA0010A102003E01F00E0200200600010000040F01430000050F4C0F02003E0610A1E7
:2059EA0002003E01F50E0200200620010000040F02430000050F4C0F02003E0610A1020050
:205A0A003E01FA0E0200200640010000040F03430000050F4C0F02003E0610A102003E01CC
:205A2A00FF0E0200200660010000040F04430000050F4C0F02003E0610A102003E01040FB2
:205A4A000200200680010000040F05430000050F4C0F02003E0610A102003E01090F020077
:205A6A002006A0010000040F06430000050F4C0F02003E0610A102003E010E0F020020060D
:205A8A00C0010000040F07430000050F4C0F02003E0610A102003E01130F02002006E0010C
:205AAA000000040F08430000050F4C0F02003E0610A102003E01180F020020060002000086
:205ACA00040F09430000050F4C0F02003E0610A102003E011D0F0200200620020000040F2D
:205AEA000A430000050F4C0F02003E0610A102003E01220F0200200640020000040F0B43AC
:205B0A000000050F4C0F02003E0610A102003E01270F0200200660020000040F0C430000B2
:205B2A00050F4C0F02003E0610A102003E012C0F0200200680020000040F0D430000050F58
:205B4A004C0F02003E0610A102003E01310F02002006A0020000040F0E430000050F4C0FCB
:205B6A0002003E0610A102003E01360F02002006C0020000040F0F430000050F4C0F0200DE
:205B8A003E0610A102003E013B0F02002006E0020000040F10430000050F4C0F02003E0656
:205BAA0010A102003E01400F0200200600030000040F11430000050F4C0F02003E0610A1A2
:205BCA0002003E01450F0200200620030000040F12430000050F4C0F02003E0610A102000B
:205BEA003E014A0F0200200640030000040F13430000050F4C0F02003E0660030000040F04
:205C0A0014430000050F00A302003E0100160200BE060E9E0200140F01000000240F00004A
:205C2A0000000C0F010070000411000000B48F700F0000001E0E000000003E5900007000C4
:205C4A000011000070000C11000000003E59000070000011000070000C11000000003E5960
:205C6A00000070000011000070000C11000000003E59000070000011000070000C11000067
:205C8A0000003E59000070000011000070000C110100700005110000700008113A8C02007D
:205CAA00140F000000923F7000000000340F000000203F0400000000240F000000003E5906
:205CCA0000000100010F010004003E01FFFF0000010F120204003E01021004003E010000AB
:205CEA0000803E5900100000010F00420000000F01007000001100007000011100420000CC
:205D0A00000F010070000011000070000110101102003E01750F0200200601000000010F48
:205D2A00328C0200011100430000000F010070000011000070000111D81502003E060000FE
:205D4A000000340F00160200BE0601430000010F010070000111000070000811000070004A
:205D6A00081100007000081100007000081100007000081100007000081100007000081153
:205D8A0000007000081100007000081100007000081100007000081100007000081100004C
:205DAA007000081100007000081100007000081100007000081100007000081100007000BC
:205DCA00081100007000081100007000081101000000240F000000000C0F00010000040F2B
:205DEA00EC150200BE0620010000040FEC150200BE0640010000040FEC150200BE0660015B
:205E0A000000040FEC150200BE0680010000040FEC150200BE06A0010000040FEC1502008C
:205E2A00BE06C0010000040FEC150200BE06E0010000040FEC150200BE0600020000040F29
:205E4A00EC150200BE0620020000040FEC150200BE0640020000040FEC150200BE066002F7
:205E6A000000040FEC150200BE0680020000040FEC150200BE06A0020000040FEC1502002A
:205E8A00BE06C0020000040FEC150200BE06E0020000040FEC150200BE0600030000040FC6
:205EAA00EC150200BE0620030000040FEC150200BE0640030000040FEC150200BE06600394
:205ECA000000040FEC150200BE063A8C0200140F00000000340F01000000240F000000007C
:205EEA00250FFFFF0000010F120204003E0100000100010F14000000680F040000001E0E33
:205F0A00000000007E59010004003E01021004003E01000000803E5900100000010F00428E
:205F2A000000000F01007000001100007000011100420000000F0100700000110000700001
:205F4A000110101102003E01D30F0200200601000000010F328C0200011100430000000F85
:205F6A00010070000011000070000111D81502003E06478D02000010488D02000210001100
:205F8A0002003E0168100200000610A102003E01E70F0200200680030000040F1543000038
:205FAA00050F341002003E0610A102003E01EC0F02002006A0030000040F16430000050F01
:205FCA00341002003E0610A102003E01F10F02002006C0030000040F17430000050F34108B
:205FEA0002003E0610A102003E01F60F02002006E0030000040F18430000050F3410020087
:20600A003E0610A102003E01FB0F0200200600040000040F19430000050F341002003E06FD
:20602A0010A102003E0100100200200620040000040F1A430000050F341002003E0610A149
:20604A0002003E0105100200200640040000040F1B430000050F341002003E0610A10200B2
:20606A003E010A100200200660040000040F1C430000050F341002003E0610A102003E012F
:20608A000F100200200680040000040F1D430000050F341002003E0610A102003E01141004
:2060AA0002002006A0040000040F1E430000050F341002003E0610A102003E0119100200DB
:2060CA002006C0040000040F1F430000050F341002003E0610A102003E011E100200200671
:2060EA00E0040000040F20430000050F341002003E0610A102003E0123100200200600054C
:20610A000000040F21430000050F341002003E0610A102003E0128100200200620050000E9
:20612A00040F22430000050F341002003E0610A102003E012D100200200640050000040F90
:20614A0023430000050F341002003E0610A102003E0132100200200660050000040F2443F6
:20616A000000050F341002003E0680050000040F25430000050F00A302003E01010070000E
:20618A00041100160200BE060E9E0200140F01000000240F000000000C0F000000B48F7031
:2061AA000F0000001E0E000000003E59000070000011000070000C11000000003E5900005E
:2061CA0070000011000070000C11000000003E59000070000011000070000C110000000002
:2061EA003E59000070000011000070000C11000000003E59000070000011000070000C114B
:20620A000100700005110000700008114E8C0200140F000000923F7000000000340F0000E1
:20622A0000203F0400000000240F000000003E5900000100010F010004003E01FFFF0000D4
:20624A00010F120204003E01021004003E01000000803E5900100000010F00420000000FF0
:20626A0001007000001100007000011100420000000F01007000001100007000011010119B
:20628A0002003E015D100200200601000000010F328C0200011100430000000F0100700078
:2062AA000011000070000111D81502003E0600000000340F00160200BE0615430000010F87
:2062CA0001007000011100007000081100007000081100007000081100007000081100000D
:2062EA00700008110000700008110000700008110000700008110000700008110000700077
:20630A000811000070000811000070000811000070000811000070000811000070000811AD
:20632A0000007000081100007000081101000000240F000000000C0F80030000040FEC155B
:20634A000200BE06A0030000040FEC150200BE06C0030000040FEC150200BE06E003000070
:20636A00040FEC150200BE0600040000040FEC150200BE0620040000040FEC150200BE065D
:20638A0040040000040FEC150200BE0660040000040FEC150200BE0680040000040FEC15FF
:2063AA000200BE06A0040000040FEC150200BE06C0040000040FEC150200BE06E00400000D
:2063CA00040FEC150200BE0600050000040FEC150200BE0620050000040FEC150200BE06FB
:2063EA0040050000040FEC150200BE0660050000040FEC150200BE0680050000040FEC159C
:20640A000200BE064E8C0200140F00000000340F01000000240F00000000250FFFFF000004
:20642A00010F120204003E0100000100010F11000000680F040000001E0E000000007E594B
:20644A00010004003E01021004003E01000000803E5900100000010F00420000000F010010
:20646A007000001100007000011100420000000F0100700000110000700001101011020098
:20648A003E01B2100200200601000000010F328C0200011100430000000F01007000001112
:2064AA00000070000111D81502003E0646534821020F212200003E01C6100200200600107A
:2064CA000000010F00420000000F010070000011000070000111F9090200BE06D815020096
:2064EA003E0646535421020F212200003E01F21002002006468D02000110101102003E013B
:20650A00DF1002002006478D02000110488D0200021010A102003E01000000921F700A422B
:20652A000000000F011100003E010100700001110000700002113A8C0200140F0000000000
:20654A00340F000000203F0400000000240F000000003E59FFFF0000010F010004003E016F
:20656A00221000003E02021004003E01000000803E59D81502003E06478D02000110488D44
:20658A000200021010A102003E01000000921F701E420000000F011100003E010100700099
:2065AA0001110000700002114E8C0200140F00000000340F000000203F0400000000240F64
:2065CA00000000003E59FFFF0000010F010004003E01221000003E02021004003E01000001
:2065EA0000803E59D81502003E0646545021020F212200003E01FC1002002006468D0200A0
:20660A000110101102003E01FA1002000006040000000014FB1002003E060400000020144A
:20662A00D81502003E0647454E21020F212200003E010A1102002006468D020001108B8C4F
:20664A0002000111478D020001108C8C02000111488D020001108D8C02000111498D02001C
:20666A0001108A8C020001114A8D02000110918C02000111D81502003E0649445021020F78
:20668A00212200003E012D1102002006468D02000110A3A002000111478D02000110A4A0A0
:2066AA0002000111488D02000110A6A002000111498D020001101FA1020001114A8D0200E4
:2066CA00011020A1020001114B8D02000110101102003E011C11020000060800000000142C
:2066EA001D1102003E060800000020144C8D02000110101102003E01221102000006100047
:20670A0000000014231102003E06100000002014A3A002000010AEA00200011001220000C4
:20672A003E01B2ED0200021120A202003E01B1ED02000211A4A00200001000A002003E016F
:20674A00B3ED02000011D81502003E064C454421020F212200003E01331102002006468D81
:20676A0002000110868C02000111D81502003E064D445421020F212200003E013E110200B9
:20678A002006328C0200011001000000020F122104003E0100430000000F0100700000119C
:2067AA00000070000111328C02000111D81502003E064E434621020F212200003E01541158
:2067CA0002002006468D0200150F00000000350F01000000240F00000000250F0000800062
:2067EA003E5BA9A00200011182EB02000111DAA00200140F00000000340F10000000680FAF
:20680A00020000001E0E000080003E5B000080803E59EAA00200140F10000000680F020058
:20682A0000001E0E000080003E5B000080803E59D81502003E064E434E21020F21220000EB
:20684A003E0102120200200600000000010F328C02000111468D020001109FA00200011198
:20686A0010A102003E01641102002406FEFFFFFF030F00040000000FFEFFFFFF040FFFFF4F
:20688A00FFFF050FE91102043E06F00A0000010FF00A0000020F10A102003E016D11020011
:2068AA002406FCFFFFFF030F00020000000FFEFFFFFF040FFDFFFFFF050FE91102043E0628
:2068CA0078050000010F78050000020F10A102003E01761102002406F8FFFFFF030F540192
:2068EA000000000FFAFFFFFF040FFDFFFFFF050FE91102043E06A5030000010FA5030000C3
:20690A00020F10A102003E017F110200240600010000000FF0FFFFFF030FFAFFFFFF040F95
:20692A00F5FFFFFF050FE91102043E06BC020000010FBC020000020F10A102003E018811DB
:20694A0002002406E0FFFFFF030FC8000000000FEAFFFFFF040FF5FFFFFF050FE91102043B
:20696A003E0630020000010F30020000020F10A102003E01911102002406C0FFFFFF030FB5
:20698A00AA000000000FEAFFFFFF040FD5FFFFFF050FE91102043E06D1010000010FD1015C
:2069AA000000020F10A102003E019A110200240680FFFFFF030F91000000000FAAFFFFFF1D
:2069CA00040FD5FFFFFF050FE91102043E0690010000010F90010000020F10A102003E013B
:2069EA00A3110200240680000000000F00FFFFFF030FAAFFFFFF040F55FFFFFF050FE911F5
:206A0A0002043E065E010000010F5E010000020F10A102003E01AC110200240600FEFFFF6C
:206A2A00030F71000000000FAAFEFFFF040F55FFFFFF050FE91102043E0637010000010F0F
:206A4A0037010000020F10A102003E01B5110200240600FCFFFF030F66000000000FAAFED6
:206A6A00FFFF040F55FDFFFF050FE91102043E0618010000010F18010000020F10A102004D
:206A8A003E01BE11020024065D000000000F00F8FFFF030FAAFAFFFF040F55FDFFFF050F25
:206AAA00E91102043E06FE000000010FFE000000020F10A102003E01C7110200240600F085
:206ACA00FFFF030F55000000000FAAFAFFFF040F55F5FFFF050FE91102043E06E9000000FA
:206AEA00010FE9000000020F10A102003E01D0110200240600E0FFFF030F4E000000000F36
:206B0A00AAEAFFFF040F55F5FFFF050FE91102043E06D7000000010FD7000000020F10A1A6
:206B2A0002003E01D9110200240600C0FFFF030F49000000000FAAEAFFFF040F55D5FFFFFF
:206B4A00050FE91102043E06C8000000010FC8000000020F10A102003E01E2110200240611
:206B6A0044000000000F0080FFFF030FAAAAFFFF040F55D5FFFF050FE91102043E06BA0089
:206B8A000000010FBA000000020F40000000000F0000FFFF030FAAAAFFFF040F5555FFFFA4
:206BAA00050FE91102043E06AF000000010FAF000000020FFAA002000111FEA00200001195
:206BCA00FDA002000011FBA00200021100000000000F001002003E01FB11020000060100D6
:206BEA000000000F001002003E01F71102000006A9A002000010041004003E01A9A002001E
:206C0A000011FE1102003E06A9A002000010051004003E01A9A002000011FE1102003E06A0
:206C2A00A9A002000010031004003E01A9A002000011F9090200BE0601000000010F328CA6
:206C4A0002000111D81502003E064E455221020F212200003E010D12020020060000000003
:206C6A00010F328C02000111468D02000110A0A002000111F9090200BE0601000000010F15
:206C8A00328C02000111D81502003E064E524621020F212200003E012912020020060000E8
:206CAA000000010F328C02000111468D020001109EA00200011110A102003E011912020091
:206CCA002006251202043E06F00A0000010FFCA00200011110A102003E011E1202002006FF
:206CEA00251202043E0678050000010FFCA00200011110A102003E01231202002006251246
:206D0A0002043E06A5030000010FFCA002000111BC020000010FFCA002000111F909020035
:206D2A00BE0601000000010F328C02000111D81502003E064F52533F020F212200003E01A9
:206D4A003B12020020060B000000000F659502000011F9EC0200140F00000000340F04003C
:206D6A000000240F64950200110F00000000310F000000603E0401000000240F1400000091
:206D8A00680F020000001E0E000080003E59000080803E53D1150200BE06C21502003E06D3
:206DAA005244593F020F212200003E014A1202002006D1150200BE0652445921010F6895BB
:206DCA000200011111F000783E026995020001110A000000010F6A9502000111000000009D
:206DEA00010F6B950200011103000000000F659502000011C21502003E0652454621020F1A
:206E0A00212200003E018A120200200600000000000F328C02000011B1A00200100F0000D0
:206E2A000000300FB2A002000011B3A002000011B4A002000011B5A002000011010000006E
:206E4A00010F468D02002110CAA002002111000080807E40478D02002110CBA00200211110
:206E6A00000080807E40488D02002110CCA002002111000080807E40498D02002110CDA06E
:206E8A0002002111000080807E404A8D02002110CEA002002111000080807E404B8D0200B2
:206EAA002110CFA002002111000080807E404C8D02002110D0A002002111000080807E40C8
:206ECA004D8D02002110D1A002002111000080807E404E8D02002110D2A002002111000084
:206EEA0080807E404F8D02002110D3A002002111000080807E40508D02002110D4A00200D0
:206F0A002111000080807E40518D02002110D5A002002111000080807E40528D02002110ED
:206F2A00D6A002002111000080807E40538D02002110D7A002002111000080807E40548D82
:206F4A0002002110D8A002002111000080807E40558D02002110D9A00200211100008080C8
:206F6A007E40F9090200BE0601000000010F328C02000111D81502003E06524E5021020F49
:206F8A00212200003E01901202002006468D02000110BA8C02000111D81502003E06525383
:206FAA005421020F212200003E01B0120200200600000000010F328C0200011100430000B0
:206FCA00000F01007000001100007000011100420000000F01007000001100100000010FA1
:206FEA00000070000111468D02000110101102003E01A0120200200699EB02000111478D77
:20700A0002000110101102003E01A412020020069AEB02000111F9090200BE060042000070
:20702A00000F010070000011000070000110101102003E01A5120200200601000000010FE2
:20704A00328C0200011100430000000F010070000011000070000111D81502003E06534137
:20706A004D21020F212200003E01731302002006468D02000110478D02000210488D0200B2
:20708A00031000430000000F01007000001100000000000F000070000011328C020000119E
:2070AA0058140000000F012400003E01C81202002006878C0200001151C80000000FABC22A
:2070CA00A245010F201202003E013D1302000006ABC22244010F301302003E013D1302002B
:2070EA000006ABC2A242010F3D1302003E066A180000000F012400003E01D5120200200685
:20710A00878C020000115FC80000000F0050C345010F201202003E013D1302000006005086
:20712A004344010F301302003E013D13020000060050C342010F3D1302003E06CA1F0000EE
:20714A00000F012400003E01E21202002006878C0200001150C80000000F2B50FE45010F7B
:20716A00201202003E013D13020000062B507E44010F301302003E013D13020000062B5096
:20718A00FE42010F3D1302003E0626260000000F012400003E01EF1202002006878C020002
:2071AA0000115EC80000000F80961846010F201202003E013D130200000680969844010F2E
:2071CA00301302003E013D130200000680961843010F3D1302003E06B1280000000F0124A5
:2071EA0000003E01FC1202002006878C0200001153C80000000FABC22246010F20120200A7
:20720A003E013D1302000006ABC2A244010F301302003E013D1302000006ABC22243010FAC
:20722A003D1302003E06943F0000000F012400003E01091302002006878C0200001152C8E4
:20724A000000000F2B507E46010F201202003E013D13020000062B50FE44010F30130200E9
:20726A003E013D13020000062B507E43010F3D1302003E06C1450000000F012400003E0112
:20728A00161302002006878C0200001155C80000000F49828B46010F201202003E013D13D2
:2072AA000200000649820B45010F301302003E013D130200000649828B43010F3D130200BA
:2072CA003E0661510000000F012400003E01231302002006878C0200001157C80000000F89
:2072EA00ABC2A246010F201202003E013D1302000006ABC22245010F301302003E013D139C
:20730A0002000006ABC2A243010F3D1302003E06FE6C0000000F012400003E013013020041
:20732A002006878C0200001154C80000000F92FBD946010F201202003E013D130200000645
:20734A0092FB5945010F301302003E013D130200000692FBD943010F3D1302003E06287F16
:20736A000000000F012400003E01BE1202002006878C0200001156C80000000F2B50FE4686
:20738A00010F201202003E013D130200000615008045010F301302003E013D130200000642
:2073AA002B50FE43010F3D1302003E06BB8C02000111A6050200BE06B6050200BE06B60559
:2073CA000200BE06FF0F0000040F040004003E01A6050200BE06C8000000680F02000000C3
:2073EA001E0EB6050200BE0600000000000001420000000F0100700000110000700002117F
:20740A0002420000000F010070000011000070000311888C02000211898C020003111E0097
:20742A000000040F201202003E0157130200000605000000040F301302003E015713020042
:20744A00000602000000040FAEA002000411A3A002000010AEA002000110012200003E018A
:20746A00B2ED0200021120A202003E01B1ED02000211A4A00200001000A002003E01B3EDC1
:20748A0002000011B6050200BE0651070200BE06F9090200BE0600100000010F0042000006
:2074AA00000F01007000001100007000011100420000000F0100700000110000700001105B
:2074CA00101102003E0168130200200601000000010F328C0200011100430000000F010067
:2074EA0070000011000070000111D81502003E0653444521020F212200003E01A113020006
:20750A00200694E70200110F00000000310F01000000200FAC030000680F010000001E0EDB
:20752A0000000000009200000000080F0A000000090F468D0200100F00000000300F94E7C8
:20754A000200110F00000000000F01000000010F000080811F71000000403E0417000000B5
:20756A00680F070000001E0E000000013E50201202003E018D1302000006000080803E521D
:20758A00000000813E52009002003E01109102003E01000080801F71000080883F700000D6
:2075AA0000803E52000080881F70809802003E01982000003E01811302002406000000000A
:2075CA00000F328C0200001194E70200110F2CE30200100FAC030000680F020000001E0EA0
:2075EA00000000003E52000000803E50F9090200BE0601000000000F328C02000011D8154D
:20760A0002003E065344453F020F212200003E01CF1302002006D1150200BE06CC010000E9
:20762A00000F009002003E0165950200001194E70200110F00000000310F01000000200F46
:20764A00AC030000680F010000001E0E00000000009200000000080F0A000000090F2CE3F3
:20766A000200100F00000000300F94E70200110F17000000210F000000003E50001002001C
:20768A003E01C01302000006000000821F7107000000000D000000003E5000A002003E0131
:2076AA00000000910F70000000003E50000080884F70000000503E04000000803E520000B9
:2076CA0080884F70000000483E04809802003E01982000003E01B41302002406689502000D
:2076EA00100F00000000300F94E70200110FCC010000010F04000000010D000080003E5286
:20770A00000080803E5011F000783E02000080803E50C21502003E0653445221020F21220F
:20772A0000003E01FD130200200694E70200110F00000000310F01000000200FBC000000FF
:20774A00680F010000001E0E00000000009200000000080F04000000090F468D0200100FC2
:20776A0000000000300F94E70200110F00000000000F01000000010F000080811F71000072
:20778A0000403E0417000000680F070000001E0E000000013E50201202003E01E91302009C
:2077AA000006000080803E52000000813E52009002003E01109102003E01000080801F71D5
:2077CA00000080883F70000000803E52000080881F70809802003E01982000003E01DD1301
:2077EA000200240600000000000F328C0200001194E70200110FD8E60200100FBC0000003B
:20780A00680F020000001E0E000000003E52000000803E50F9090200BE0601000000000F43
:20782A00328C02000011D81502003E065344523F020F212200003E012B1402002006D11532
:20784A000200BE06CC010000000F009002003E0165950200001194E70200110F0000000001
:20786A00310F01000000200FBC000000680F010000001E0E00000000009200000000080F85
:20788A0004000000090FD8E60200100F00000000300F94E70200110F17000000210F0000C0
:2078AA0000003E50001002003E011C1402000006000000821F7107000000000D0000000081
:2078CA003E5000A002003E01000000910F70000000003E50000080884F70000000503E0438
:2078EA00000000803E52000080884F70000000483E04809802003E01982000003E011014A9
:20790A000200240668950200100F00000000300F94E70200110FCC010000010F0400000056
:20792A00010D000080003E52000080803E5011F000783E02000080803E50C21502003E062D
:20794A005349443F020F212200003E013E1402002006D1150200BE064E4F5641010F689504
:20796A000200011111F000783E0269950200011143533220010F6A950200011111F000789A
:20798A003E026B950200011153445320010F6C950200011111F000783E026D95020001118B
:2079AA0004000000000F659502000011C21502003E0653465121020F212200003E01551479
:2079CA0002002006468D020001108E8C02000111478D020001108F8C02000111488D020074
:2079EA000110908C02000111498D02000110B48C020001114A8D02000110B58C02000111C0
:207A0A004B8D02000110B68C020001110A8D02000110B7ED0200011100000000010F0A8D12
:207A2A000200011151070200BE06B7ED020001100A8D02000111D81502003E06534D502164
:207A4A00020F212200003E0169140200200677BE7F3F030F468D02000110312408003E015D
:207A6A005D140200220677BE7F3F010FB78C02000111478D02000110312408003E0162140E
:207A8A000200220677BE7F3F010FB88C02000111488D02000110312408003E016714020056
:207AAA00220677BE7F3F010FB98C02000111D81502003E0653524321020F212200003E0169
:207ACA00741402002006468D020001100A000000000F012000003E0172140200200684ED6E
:207AEA000200001186ED02000011928C02000111D81502003E065354533F020F21220000F1
:207B0A003E01C21402002006D1150200BE06A8A00200011068950200011111F000783E024D
:207B2A00699502000111A7A0020001106A950200011111F000783E026B95020001110000EF
:207B4A000000010FA8A002000111A7A00200011182ED020001106C950200011111F0007844
:207B6A003E026D950200011100000000010F82ED020001110000200080148C1402003A067C
:207B8A0001000000010F6E950200011111F000783E026F950200011100002000201482EB21
:207BAA000200011070950200011111F000783E0271950200011100000000010F00000001AB
:207BCA008014981402003A0601000000010F72950200011111F000783E0273950200011118
:207BEA000000000120149BED0200011074950200011111F000783E027595020001110000B7
:207C0A000000010F9BED02000111ADA00200011076950200011111F000783E027795020068
:207C2A00011100000000010FADA002000111000000048014AB1402003A0601000000010F0D
:207C4A0078950200011111F000783E02799502000111000000042014AA8C020001107A958E
:207C6A000200011111F000783E027B9502000111AB8C020001107C950200011111F0007821
:207C8A003E027D9502000111AF8C020001107E950200011111F000783E027F95020001111E
:207CAA00B08C0200011080950200011111F000783E028195020001110E000000000F659548
:207CCA0002000011C21502003E0654504221020F212200003E012015020020060000000073
:207CEA00020F468D02000110EAA002000111212100003E011E1502008206478D02000110C0
:207D0A00EBA002000111212100003E011E1502008206488D02000110ECA0020001112121B2
:207D2A0000003E011E1502008206498D02000110EDA002000111212100003E011E150200FD
:207D4A0082064A8D02000110EEA002000111212100003E011E15020082064B8D02000110DC
:207D6A00EFA002000111212100003E011E15020082064C8D02000110F0A002000111212146
:207D8A0000003E011E15020082064D8D02000110F1A002000111212100003E011E15020095
:207DAA0082064E8D02000110F2A002000111212100003E011E15020082064F8D0200011070
:207DCA00F3A002000111212100003E011E1502008206508D02000110F4A0020001112121DA
:207DEA0000003E011E1502008206518D02000110F5A002000111212100003E011E1502002D
:207E0A008206528D02000110F6A002000111212100003E011E1502008206538D0200011003
:207E2A00F7A002000111212100003E011E1502008206548D02000110F8A00200011121216D
:207E4A0000003E011E1502008206558D02000110F9A002000111212100003E011E150200C4
:207E6A008206ACA002000211003402001C0F000000003C0F003402001D0F000000003D0FB5
:207E8A00010000002C0FFEA002002D1000000081DF7200000000030FEAA00200140F00002C
:207EAA000000340F01000000240F9FA002006810090000001E0E000080003E5900000097A5
:207ECA001F70000000307F04212100003E0101000000010D000080813F59000000687F0442
:207EEA0000008080DF710000008E1F70D81502003E06000000811F70000000003E0A5450DC
:207F0A004621020F212200003E017C150200200600000000020F468D02000110DAA0020031
:207F2A000111212100003E011E1502008206478D02000110DBA002000111212100003E01F0
:207F4A001E1502008206488D02000110DCA002000111212100003E011E1502008206498DCE
:207F6A0002000110DDA002000111212100003E011E15020082064A8D02000110DEA00200AB
:207F8A000111212100003E011E15020082064B8D02000110DFA002000111212100003E0188
:207FAA001E15020082064C8D02000110E0A002000111212100003E011E15020082064D8D62
:207FCA0002000110E1A002000111212100003E011E15020082064E8D02000110E2A002003F
:207FEA000111212100003E011E15020082064F8D02000110E3A002000111212100003E0120
:20800A001E1502008206508D02000110E4A002000111212100003E011E1502008206518DF5
:20802A0002000110E5A002000111212100003E011E1502008206528D02000110E6A00200D2
:20804A000111212100003E011E1502008206538D02000110E7A002000111212100003E01B7
:20806A001E1502008206548D02000110E8A002000111212100003E011E1502008206558D89
:20808A0002000110E9A002000111212100003E011E1502008206ABA0020002110030020056
:2080AA001C0F000000003C0F003002001D0F000000003D0F010000002C0FFEA002002D107D
:2080CA0000000081DF7200000000030FDAA00200140F00000000340F01000000240F9FA05D
:2080EA0002006810090000001E0E000080003E59000000971F70000000307F042121000095
:20810A003E0101000000010D000080813F59000000687F0400008080DF710000008E1F7016
:20812A00D81502003E0655535421020F212200003E01861502002006468D020001100000A9
:20814A0000810F770000FFFF030F230204003E01121204003E01000000B82F70D8150200E9
:20816A003E0657475421020F212200003E01C21502002006468D02000010478D0200011040
:20818A00488D02000210498D020003104A8D0200041000A002003E01A7150200000600006F
:2081AA000000050F00004200180F00000000380F01000000280FFDA002002D10800000005D
:2081CA002F0F509502003E01452700003E01A115020000069FA002006810010000001E0EE2
:2081EA00000000287E04000000387E04000000387E04000000387E04000000387E04961538
:20820A0002003E0630A302003E01B31502000006000000B43F70010000001E0E0000002872
:20822A007E04B31502003E06101102003E0100300200180FAD150204000600000000380FD4
:20824A0001000000280F00340200180F30A302003E01B31502000006FEA0020029100000C2
:20826A0000B43F70010000001E0E000000087E04000000B42F70209402003E016595020096
:20828A00041104000000240F64950200110F00000000310F000000603E0401000000210F5A
:2082AA00040000001E0E000080003F50000080807E5211F000783E02000080807E52D11536
:2082CA000200BE06C21502003E0664950200000F78000000001101000000000F7900000095
:2082EA00001120080000000F7A000000001100000000030FF0000000031100000000000F7C
:20830A00899D02000011859D02000310F00000000311000000043E0A00000000000F849D63
:20832A000200001101000000000F64950200001143310000010F669502000111000000046D
:20834A003E0A50430000010F679502000111D1150200BE06BFED020001106895020001119C
:20836A0011F000783E02699502000111204F4B0A010F6A950200011111F000783E026B9588
:20838A000200011103000000000F659502000011C21502003E0668950200011111F00078F9
:2083AA003E02699502000111D1150200BE0602000000000F659502000011C21502003E067A
:2083CA00E41502003E060100700004110E9E0200140F000000B48F700F0000001E0E00000F
:2083EA0000003E59000070000011000070000C11000000003E590000700000110000700046
:20840A000C11000000003E59000070000011000070000C11000000003E5900007000001178
:20842A00000070000C11000000003E59000070000011000070000C11000000003E0AFF00B9
:20844A0000000C0F2C0C04003E01CE9D0200140F00000092CF70000000203F0400000004B4
:20846A003E598E9D0200140F000000203F04000000003E590000008A0F7001000000240FD4
:20848A000E9E0200100F00000000300F000000B48F700A0000001E0E000000003E59000046
:2084AA0000803E51000000003E59000000803E51000000003E59000000803E510000000057
:2084CA003E59000000803E51000000003E59000000803E5100FF00000C0F2C0C04003E01B1
:2084EA00CCF800783E02CE9D0200140F00000092CF70000000203F04000000063E598C18F1
:20850A0000003E018E9D0200140F000000203F04000000003E590000008A0F7001000000BE
:20852A00240F000000B4CF700A0000001E0E000000003E59000000803E51000000003E5998
:20854A00000000803E51000000003E59000000803E51000000003E59000000803E510000B6
:20856A0000003E59000000803E51000000003E0A9FA002000410402400003E01000000000B
:20858A00020A00300200180F00000000380F01000000280FFEA00200291000A402003E012F
:2085AA003F1602000006000000B44F70010000001E0E000000087E0400000000040F000017
:2085CA0000B49F72010000001E0E000000823F5000340200180F00A402003E0149160200EB
:2085EA000006000000B44F70010000001E0E000000087E0400000000040F000000B49F7269
:20860A00010000001E0E000000823F50F00A0000340F56AC0200440F46B70200141001005A
:20862A000000240FFAA00200251000A402003E01571602000006000000B44F70010000005E
:20864A001E0E000000283F04000000B49F72010000001E0E000000000099000000003E0AA6
:20866A00000007000A14008000002A14000070002C14D5070200BE0601000000000F8041EA
:20868A000000010F010070000111000070000110012100003E016016020020066620000037
:2086AA00000F00420000010F010070000111000070000011FC040200BE0601000000000F75
:2086CA00001002003E016E1602000006791D0200BE0601000000010F328C02000111004331
:2086EA000000000F010070000011000070000111928C020001100A000000000F01200000F2
:20870A003E017C1602000006C1050200BE06849D02000010001002003E01230B0200A00690
:20872A00731602003E06010000008014A91602003A06C1ED02007011000010000014000075
:20874A000800201402000000201400000000000FC2ED02000011C1050200BE06849D02001D
:20876A000010001002003E01230B0200A006000002000014000002008014891602001A064B
:20878A0057040200BE067E1A0200BE06C2ED02000010009002003E01C2ED02000011C80034
:2087AA000000010F012000003E01841602002006000010002014000008000014000000001D
:2087CA00000FC2ED02000011C1050200BE06849D02000010001002003E01230B0200A006D8
:2087EA000000020000140000020080149C1602001A0657040200BE067E1A0200BE06C2EDC1
:20880A0002000010009002003E01C2ED02000011C8000000010F012000003E0197160200C2
:20882A002006C1ED02007010000008000014000010000014C1050200BE06849D02000010D9
:20884A00001002003E01230B0200A006928C020001100A000000000F012000003E01A9167E
:20886A0002002006010000008014E11602003A06F8EC02000010009002003E01F8EC02004B
:20888A000011A6A002000110102100003E01E1160200240600000000020FF8EC02000211C7
:2088AA00020000008014D71602003A06F7EC02000010009002003E01F7EC02000011A5A0E8
:2088CA0002000110102100003E01D71602002406F7EC0200021100000600001400000600DA
:2088EA008014C51602001A0657040200BE0695040200BE067E1A0200BE0681EB0200001081
:20890A00A7A00200001100000000000F81EB02000011849D02000010001002003E01230BB3
:20892A000200A006F31B0200BE0680EB02000010A8A00200001100000000000F80EB02005D
:20894A000011A91602003E06000002000014000002008014D81602001A0657040200BE061A
:20896A007E1A0200BE0681EB02000010A7A00200001100000000000F81EB02000011A9166A
:20898A0002003E06020000008014F51602003A06F7EC02000010009002003E01F7EC0200F9
:2089AA000011A5A002000110102100003E01F5160200240600000000020FF7EC0200021194
:2089CA00000004000014000004008014EC1602001A0695040200BE06F31B0200BE0680EB1B
:2089EA0002000010A8A00200001100000000000F80EB02000011A91602003E06000001006D
:208A0A000014000001008014F61602001A06A91602003E06C4ED0200140F00000000340F57
:208A2A000000803F070F00088B087E6800100A828F7070270A000201410413003E0140912F
:208A4A000C003E01010033003E0270270A00300110A40C003E01000080087E68140C930853
:208A6A007E68401C59003E01C128080A7E68800C0B003E01C42408868F70121702000206B3
:208A8A00CC0C130A7E6802000006000CC40493087E68141408003E01C40413003E014804BF
:208AAA0013043E0A481C08003E01C70013003E01000000003E0AAA8C02000010D1ED020039
:208ACA000011AB8C02000010D2ED02000011AF8C02000010D3ED02000011B08C02000010F2
:208AEA00D4ED02000011C48C0200100F00000000300F348C0200110F00000000310F0100C5
:208B0A000000210F80000000680F020000001E0E000000007E50000000807E52AAA002008C
:208B2A000010000000B80F70000010000014000008000014A3A002000010AEA002000110EE
:208B4A00012200003E01B2ED0200021120A202003E01B1ED02000211A4A00200001000A049
:208B6A0002003E01B3ED020000111DA102000010A3EB0200100FA0000000680F0100000060
:208B8A001E0E000000803E501DA1020000100000803E010F010013003E0143EC0200100F50
:208BAA00A0000000680F010000001E0E000000803E501DA1020000101EA1020001100100B6
:208BCA0013003E010000803F010F102108003E0183EB020001110DED0200100F0000000055
:208BEA00300F01000000200F14000000680F010000001E0E000080803E500B100000000F8C
:208C0A00358C0200001104000000000FAC8C0200001109000000000FAD8C020000110A00AA
:208C2A000000000FAE8C020000110A000000000F368C0200001109000000000F378C020003
:208C4A00001166000000000FB38C0200001101000000000FA98C02000011D1ED020000100A
:208C6A00AA8C02000011D2ED02000010AB8C02000011D3ED02000010AF8C02000011D4EDA5
:208C8A0002000010B08C0200001100000080AF77000000C0010F010104003E0111E2007843
:208CAA003E02B18C0200011100000030010F010104003E0111E400783E02B28C0200011195
:208CCA00DAA00200100F00000000300F01000000200F00000000000F10000000680F0500E5
:208CEA0000001E0E000080003E50102200003E01751702000406000000801F700000000018
:208D0A000000ABA002000011EAA00200100F00000000000F10000000680F050000001E0E79
:208D2A00000080003E50102200003E017F1702000406000000801F70000000000000ACA0AD
:208D4A0002000011CAA00200100F01000000010F10000000680F0F0000001E0E0000000098
:208D6A003E5000A002003E018A1702002006B2A002000111931702003E0600A002003E017A
:208D8A008E1702002006B3A002000111931702003E0600A002003E01921702002006B4A09F
:208DAA0002000111931702003E06B5A00200011100000000000000002000201400004000A8
:208DCA00201400008000201400000001201400000002201400000004201400000000000FEF
:208DEA0080EB0200001181EB02000011F7EC02000011F8EC0200001149ED0200001182EDC7
:208E0A00020000114BED020000119BED02000011A7A002000011A8A00200001184ED020027
:208E2A00001186ED02000011A0EB020000114AED02000011A9A00200011082EB02000111CC
:208E4A009FA00200011010A102003E01B51702002406FEFFFFFF030F00040000000FFEFFAF
:208E6A00FFFF040FFFFFFFFF050F3A1802043E06F00A0000010FF00A0000020F10A1020063
:208E8A003E01BE1702002406FCFFFFFF030F00020000000FFEFFFFFF040FFDFFFFFF050F50
:208EAA003A1802043E0678050000010F78050000020F10A102003E01C71702002406F8FFFE
:208ECA00FFFF030F54010000000FFAFFFFFF040FFDFFFFFF050F3A1802043E06A5030000B8
:208EEA00010FA5030000020F10A102003E01D0170200240600010000000FF0FFFFFF030F8B
:208F0A00FAFFFFFF040FF5FFFFFF050F3A1802043E06BC020000010FBC020000020F10A14D
:208F2A0002003E01D91702002406E0FFFFFF030FC8000000000FEAFFFFFF040FF5FFFFFF18
:208F4A00050F3A1802043E0630020000010F30020000020F10A102003E01E21702002406BB
:208F6A00C0FFFFFF030FAA000000000FEAFFFFFF040FD5FFFFFF050F3A1802043E06D10111
:208F8A000000010FD1010000020F10A102003E01EB170200240680FFFFFF030F9100000094
:208FAA00000FAAFFFFFF040FD5FFFFFF050F3A1802043E0690010000010F90010000020F19
:208FCA0010A102003E01F4170200240680000000000F00FFFFFF030FAAFFFFFF040F55FFB2
:208FEA00FFFF050F3A1802043E065E010000010F5E010000020F10A102003E01FD170200D2
:20900A00240600FEFFFF030F71000000000FAAFEFFFF040F55FFFFFF050F3A1802043E06D3
:20902A0037010000010F37010000020F10A102003E0106180200240600FCFFFF030F6600E7
:20904A000000000FAAFEFFFF040F55FDFFFF050F3A1802043E0618010000010F18010000FC
:20906A00020F10A102003E010F18020024065D000000000F00F8FFFF030FAAFAFFFF040F67
:20908A0055FDFFFF050F3A1802043E06FE000000010FFE000000020F10A102003E01181887
:2090AA000200240600F0FFFF030F55000000000FAAFAFFFF040F55F5FFFF050F3A180204AD
:2090CA003E06E9000000010FE9000000020F10A102003E0121180200240600E0FFFF030F08
:2090EA004E000000000FAAEAFFFF040F55F5FFFF050F3A1802043E06D7000000010FD700AE
:20910A000000020F10A102003E012A180200240600C0FFFF030F49000000000FAAEAFFFF1A
:20912A00040F55D5FFFF050F3A1802043E06C8000000010FC8000000020F10A102003E0197
:20914A0033180200240644000000000F0080FFFF030FAAAAFFFF040F55D5FFFF050F3A18B8
:20916A0002043E06BA000000010FBA000000020F40000000000F0000FFFF030FAAAAFFFF55
:20918A00040F5555FFFF050F3A1802043E06AF000000010FAF000000020FFAA0020001112D
:2091AA00FEA002000011FDA002000011FBA0020002119EA00200011010A102003E014418F5
:2091CA0002002006501802043E06F00A0000010FFCA00200011110A102003E01491802009C
:2091EA002006501802043E0678050000010FFCA00200011110A102003E014E1802002006D0
:20920A00501802043E06A5030000010FFCA002000111BC020000010FFCA0020001110000AC
:20922A000000000F001002003E015E180200000601000000000F001002003E015A18020071
:20924A000006A9A002000010041004003E01A9A002000011611802003E06A9A002000010D6
:20926A00051004003E01A9A002000011611802003E06A9A002000010031004003E01A9A077
:20928A0002000011F9090200BE06EF8C020003105F8C02000311F18C02000410618C0200D6
:2092AA000411F38C02000510638C02000511F58C02000610658C02000611F78C02000710B3
:2092CA00678C020007116E1A0200BE06B6050200BE06B6050200BE0600010000000FF08C9B
:2092EA0002000310031304003E01608C02000311F28C02000410041404003E01628C020015
:20930A000411F48C02000510051504003E01648C02000511F68C02000610061604003E0139
:20932A00668C02000611F88C02000710071704003E01688C020007116E1A0200BE06B60503
:20934A000200BE06B6050200BE0600060000000F038D02000310031304003E01738C0200A8
:20936A000311058D02000410041404003E01758C02000411078D02000510051504003E01AC
:20938A00778C02000511098D02000610061604003E01798C020006110B8D020007100717AE
:2093AA0004003E017B8C020007116E1A0200BE06B6050200BE06B6050200BE0600070000E8
:2093CA00000F048D02000310031304003E01748C02000311068D02000410041404003E015B
:2093EA00768C02000411088D02000510051504003E01788C020005110A8D0200061006165A
:20940A0004003E017A8C020006110C8D02000710071704003E017C8C020007116E1A020021
:20942A00BE06B6050200BE06B6050200BE06178D02000110878C02000111188D02000210C5
:20944A00888C02000211198D02000310898C0200031158140000000F012400003E01BB1841
:20946A0002002006878C0200001151C80000000FABC2A245010F201202003E01301902004A
:20948A000006ABC22244010F301302003E01301902000006ABC2A242010F301902003E0614
:2094AA006A180000000F012400003E01C81802002006878C020000115FC80000000F0050F9
:2094CA00C345010F201202003E0130190200000600504344010F301302003E0130190200F0
:2094EA0000060050C342010F301902003E06CA1F0000000F012400003E01D51802002006F7
:20950A00878C0200001150C80000000F2B50FE45010F201202003E013019020000062B50E7
:20952A007E44010F301302003E013019020000062B50FE42010F301902003E0626260000D4
:20954A00000F012400003E01E21802002006878C020000115EC80000000F80961846010F8D
:20956A00201202003E0130190200000680969844010F301302003E01301902000006809630
:20958A001843010F301902003E06B1280000000F012400003E01EF1802002006878C020037
:2095AA00001153C80000000FABC22246010F201202003E01301902000006ABC2A244010F5A
:2095CA00301302003E01301902000006ABC22243010F301902003E06943F0000000F012434
:2095EA0000003E01FC1802002006878C0200001152C80000000F2B507E46010F2012020014
:20960A003E013019020000062B50FE44010F301302003E013019020000062B507E43010FC2
:20962A00301902003E06C1450000000F012400003E01091902002006878C0200001155C88B
:20964A000000000F49828B46010F201202003E0130190200000649820B45010F3013020011
:20966A003E0130190200000649828B43010F301902003E0661510000000F012400003E01F3
:20968A00161902002006878C0200001157C80000000FABC2A246010F201202003E013019F4
:2096AA0002000006ABC22245010F301302003E01301902000006ABC2A243010F3019020032
:2096CA003E06FE6C0000000F012400003E01231902002006878C0200001154C80000000FAA
:2096EA0092FBD946010F201202003E0130190200000692FB5945010F301302003E013019D8
:20970A000200000692FBD943010F301902003E06287F0000000F012400003E01B11802000A
:20972A002006878C0200001156C80000000F2B50FE46010F201202003E0130190200000613
:20974A0015008045010F301302003E013019020000062B50FE43010F301902003E06BB8C9E
:20976A0002000111A6050200BE06B6050200BE06B6050200BE06FF0F0000040F040004002F
:20978A003E01A6050200BE06C8000000680F020000001E0EB6050200BE0600000000000021
:2097AA0001420000000F01007000001100007000021102420000000F010070000011000073
:2097CA0070000311888C02000211898C020003111E000000040F201202003E014A1902009E
:2097EA00000605000000040F301302003E014A190200000602000000040FAEA002000411D8
:20980A00B6050200BE0651070200BE06CA8C0200021001000000030F00010000040F0143CA
:20982A000000050F3A1A0200BE06CB8C0200021002000000030F20010000040F02430000F8
:20984A00050F3A1A0200BE06CC8C0200021003000000030F40010000040F03430000050FA1
:20986A003A1A0200BE06CD8C0200021004000000030F60010000040F04430000050F3A1A1E
:20988A000200BE06CE8C0200021005000000030F80010000040F05430000050F3A1A02002D
:2098AA00BE06CF8C0200021006000000030FA0010000040F06430000050F3A1A0200BE0628
:2098CA00D08C0200021007000000030FC0010000040F07430000050F3A1A0200BE06D18C4C
:2098EA000200021008000000030FE0010000040F08430000050F3A1A0200BE06D28C020063
:20990A00021009000000030F00020000040F09430000050F3A1A0200BE06D38C020002100E
:20992A000A000000030F20020000040F0A430000050F3A1A0200BE06D48C020002100B00D2
:20994A000000030F40020000040F0B430000050F3A1A0200BE06D58C020002100C00000099
:20996A00030F60020000040F0C430000050F3A1A0200BE06D68C020002100D000000030F44
:20998A0080020000040F0D430000050F3A1A0200BE06D78C020002100E000000030FA00271
:2099AA000000040F0E430000050F3A1A0200BE06D88C020002100F000000030FC0020000B0
:2099CA00040F0F430000050F3A1A0200BE06D98C0200021010000000030FE0020000040F5A
:2099EA0010430000050F3A1A0200BE06DA8C0200021011000000030F00030000040F1143D5
:209A0A000000050F3A1A0200BE06DB8C0200021012000000030F20030000040F12430000E4
:209A2A00050F3A1A0200BE06DC8C0200021013000000030F40030000040F13430000050F8D
:209A4A003A1A0200BE06DD8C0200021014000000030F60030000040F14430000050F3A1A0A
:209A6A000200BE06DE8C0200021001000000030F80030000040F15430000050F541A020013
:209A8A00BE06DF8C0200021002000000030FA0030000040F16430000050F541A0200BE060E
:209AAA00E08C0200021003000000030FC0030000040F17430000050F541A0200BE06E18C22
:209ACA000200021004000000030FE0030000040F18430000050F541A0200BE06E28C020049
:209AEA00021005000000030F00040000040F19430000050F541A0200BE06E38C02000210F5
:209B0A0006000000030F20040000040F1A430000050F541A0200BE06E48C020002100700BC
:209B2A000000030F40040000040F1B430000050F541A0200BE06E58C02000210080000007F
:209B4A00030F60040000040F1C430000050F541A0200BE06E68C0200021009000000030F2A
:209B6A0080040000040F1D430000050F541A0200BE06E78C020002100A000000030FA00455
:209B8A000000040F1E430000050F541A0200BE06E88C020002100B000000030FC004000096
:209BAA00040F1F430000050F541A0200BE06E98C020002100C000000030FE0040000040F40
:209BCA0020430000050F541A0200BE06EA8C020002100D000000030F00050000040F2143AB
:209BEA000000050F541A0200BE06EB8C020002100E000000030F20050000040F22430000CB
:209C0A00050F541A0200BE06EC8C020002100F000000030F40050000040F23430000050F73
:209C2A00541A0200BE06ED8C0200021010000000030F60050000040F24430000050F541AD6
:209C4A000200BE06EE8C0200021011000000030F80050000040F25430000050F541A0200FF
:209C6A00BE06000000003E0AFF0000000C0F2C0C04003E01CE9D0200140F00000092CF70D8
:209C8A00000000203F04000000043E598E9D0200140F000000203F04000000003E59000072
:209CAA00008A0F7001000000240F0E9E0200100F00000000300F000000B48F700A00000094
:209CCA001E0E000000003E59000000803E51000000003E59000000803E51000000003E596B
:209CEA00000000803E51000000003E59000000803E51000000003E59000000803E5100FF00
:209D0A0000000C0F2C0C04003E01CCF800783E02CE9D0200140F00000092CF7000000020A6
:209D2A003F04000000063E598C1800003E018E9D0200140F000000203F04000000003E590C
:209D4A000000008A0F7001000000240F000000B4CF700A0000001E0E000000003E590000FC
:209D6A0000803E51000000003E59000000803E51000000003E59000000803E51000000007E
:209D8A003E59000000803E51000000003E59000000803E51000000003E0A00A302003E0141
:209DAA00010070000411071A0200BE060E9E0200140F01000000240F000000000C0F00000C
:209DCA0000B48F70030000001E0E000000003E59000070000011000070000C110100700081
:209DEA0005110000700008113A8C0200140F000000923F7000000000340F000000203F04E8
:209E0A0000000000240F000000003E5900000100010F010004003E01FFFF0000010F1202F7
:209E2A0004003E01021004003E01000000803E59000000003E0A00A302003E0101007000CC
:209E4A000411071A0200BE060E9E0200140F01000000240F000000000C0F000000B48F7029
:209E6A00030000001E0E000000003E59000070000011000070000C1101007000051100007D
:209E8A00700008114E8C0200140F000000923F7000000000340F000000203F040000000049
:209EAA00240F000000003E5900000100010F010004003E01FFFF0000010F120204003E0114
:209ECA00021004003E01000000803E59000000003E0A20410000010F0100700001110000D0
:209EEA007000031123410000010F01007000011100007000041126410000010F0100700070
:209F0A00011100007000051129410000010F0100700001110000700006112C410000010F9E
:209F2A00010070000111000070000711000000003E0A00000000300F01000000200F000055
:209F4A000000310FB2ED0200221000000000320FB6A00200130F00000000330FA4A00200A1
:209F6A002310E3EC0200140F00000000340F87ED0200150F00000000350F00000000250F5B
:209F8A0085EB0200160F00000000360F9CED0200170F00000000370F000000003A0F00009B
:209FAA0000003B0F000000003C0F000000003D0F000000003E0F000042001F0F00000000F9
:209FCA003F0F010000002C0FFDA002002D10AEA002002E10800000002F0F9FA002000B1069
:209FEA00A0A002000E1000000000050F143802000511FF2F84013E56553802001D0F00007D
:20A00A00008DFF71B2ED020006103FC02C003E01AB1A020410060000008EDF71F09F023098
:20A02A007F040000008FFF71000000B07F0402000000060D000000023F5D000000823F5994
:20A04A00000000687F04FB2C00E87F04A21A02000206A4A002000610B2A002000C10C01C0B
:20A06A0002003E01B71A020000060000008EDF710000008FFF7102000000060D00000002C8
:20A08A003F5D000000823F59000000787F04000000F87F04B3A002000C10C01C02003E01FC
:20A0AA00C11A020000060000008EDF710000008FFF7102000000060D000000023F5D000023
:20A0CA0000823F59000000787F04000000F87F04B4A002000C10C01C02003E01CB1A020070
:20A0EA0000060000008EDF710000008FFF7102000000060D000000023F5D000000823F59A6
:20A10A00000000787F04000000F87F04B5A002000C10C01C02003E01D51A02000006000038
:20A12A00008EDF710000008FFF7102000000060D000000023F5D000000823F59000000F873
:20A14A007F04FF2F04003E01553802001D0FB3ED02000210B1ED0200061048B70200110FBB
:20A16A0000000000080FCDCCCC3D090F3FC02C003E01EC1A020410060000008EDF71F09F0B
:20A18A0002307F04000000881F71000000891F71DD2D84033E50CC2C04220124020000006B
:20A1AA00060D35D9D8033E5000C85822012400C858003E018C1808003E0135D958003E01B5
:20A1CA009D1908003E01000000687F04FB2C00503E04DD1A02000206B2A002000C10C01C87
:20A1EA0002003E01FE1A02000006000000881F71000000891F710000008EDF71DD2D840354
:20A20A003E50CC2C0422012402000000020D35D9D8033E5000C85822012400C858003E0115
:20A22A008C1808583E0435D958003E019D1908003E01000000787F04B3A002000C10C01CE4
:20A24A0002003E010E1B02000006000000881F71000000891F710000008EDF71DD2D8403E2
:20A26A003E50CC2C0422012402000000020D35D9D8033E5000C85822012400C858003E01B5
:20A28A008C1808583E0435D958003E019D1908003E01000000787F04B4A002000C10C01C83
:20A2AA0002003E011E1B02000006000000881F71000000891F710000008EDF71DD2D840372
:20A2CA003E50CC2C0422012402000000020D35D9D8033E5000C85822012400C858003E0155
:20A2EA008C1808583E0435D958003E019D1908003E01000000787F04B5A002000C10C01C22
:20A30A0002003E012E1B02000006000000881F71000000891F710000008EDF71DD2D840301
:20A32A003E50CC2C0422012402000000020D35D9D8033E5000C85822012400C858003E01F4
:20A34A008C1808583E0435D958003E019D1908003E01000080869F701FA102000010000024
:20A36A000040090FD0408C830F700D0D13003E01357059003E010D0D13003E0135705900CA
:20A38A003E010D0D13003E01357059003E01070713003E01000080833E580000A040000FE3
:20A3AA00000080808F7080380E003E01812108003E014E1B02040006000000027E5B020054
:20A3CA0000000C0F409402003E014C2C00003E01531B020402060000003F020F00000000C0
:20A3EA0000000000000100149BED0200041045042C003E019BED02000411CDCCCC3D020F9A
:20A40A00531B02043E06442404003E0100000000000040A402003E01531B0204220672F9A3
:20A42A007F3F020F00000000000000000000040F000000823E5A000000003E5C0824080048
:20A44A003E01000000823E5E0000080080145A1B02001A0600000000030F553802001D0F95
:20A46A00553E02001B0FB2ED02000610FF2F04003E0148B70200110F470513003E013FC02D
:20A48A002C003E01701B020410060000008EDF71F09F02307F04000008008014701B020055
:20A4AA003A060000008FBF71000000B07F04000000881F71000000220120240C13003E0183
:20A4CA0005091322012084C858003E0102000000060D05091322012084C858843F5D0000EE
:20A4EA0000687F04000000E87E04FB2C00503E04601B02000206000010008014B51B020049
:20A50A003A06A4A002000610B2A002000C10C01C02003E01851B020000060000008EDF7182
:20A52A000000008FBF71000000881F71000000220120240C13003E0105091322012084C8C5
:20A54A0058003E0102000000060D05091322012084C858843F5D000000583E04000000780B
:20A56A007F04000000F87E04B3A002000C10C01C02003E01951B020000060000008EDF71B0
:20A58A000000008FBF71000000881F71000000220120240C13003E0105091322012084C865
:20A5AA0058003E0102000000060D05091322012084C858843F5D000000583E0400000078AB
:20A5CA007F04000000F87E04B4A002000C10C01C02003E01A51B020000060000008EDF713F
:20A5EA000000008FBF71000000881F71000000220120240C13003E0105091322012084C805
:20A60A0058003E0102000000060D05091322012084C858843F5D000000583E04000000784A
:20A62A007F04000000F87E04B5A002000C10C01C02003E01B51B020000060000008EDF71CD
:20A64A000000008FBF71000000881F71000000220120240C13003E0105091322012084C8A4
:20A66A0058003E0102000000060D05091322012084C858843F5D000000583E04FF2F040030
:20A68A003E01553E02001D0FB2ED020006103FC02C003E01C11B020410060000008EDF71B9
:20A6AA00F09F02307F040000008FAF71000000B07F0402000000060D000000023F590000BB
:20A6CA0000823F5D000000687F04FB2C00A87E04B81B02000206000010008014ED1B02008B
:20A6EA003A06A4A002000610B2A002000C10C01C02003E01CF1B020000060000008EDF7157
:20A70A000000008FAF7102000000060D000000023F59000000823F5D000000787F040000B8
:20A72A0000B87E04B3A002000C10C01C02003E01D91B020000060000008EDF710000008FDE
:20A74A00AF7102000000060D000000023F59000000823F5D000000787F04000000B87E04CD
:20A76A00B4A002000C10C01C02003E01E31B020000060000008EDF710000008FAF710200AB
:20A78A000000060D000000023F59000000823F5D000000787F04000000B87E04B5A0020058
:20A7AA000C10C01C02003E01ED1B020000060000008EDF710000008FAF7102000000060DA4
:20A7CA00000000023F59000000823F5D143802000510509502003E011438020005115E214B
:20A7EA0000003E019E1A02000206000000003E0A80EB02000010EBED02000011010000009D
:20A80A00200F00000000210F35ED0200100F00000000300F4CED0200140F00000000340FAC
:20A82A000DED0200150F00000000350F00000000360F49ED0200031082EB02000A10000091
:20A84A0000000F0FEAED02000F119FA002006810280000001E0EAFC02C003E01271C0200AB
:20A86A0030063FC02C003E011F1C02041006000000007E5000A102003E01000000003F04E4
:20A88A0082ED020001101F012C003E0182ED02000111009002003E0103000000010F012118
:20A8AA0000003E011C1C020402063F432C003E0149ED02000311000020000014EAED0200C3
:20A8CA0000100F002C003E01EAED0200001100000000020F2B1C02043E0600000000000F49
:20A8EA00000000803E502B1C02043E06000000803E50CDCC4C3E020F211C02000206000026
:20A90A0080807E50000000003E0483EB02000210F09F02003E012000000080145E1D02009A
:20A92A009A062B1C02003E06000000003E04000000003F04F09F02003E0100000000020F7A
:20A94A00000000813E5A4BED02000C1020000000040FC42C00003E01321C020002060000C4
:20A96A000000000F4BED020000110400000080143A1C02003A060DED0200150FD6ED02005E
:20A98A00160F9FA002006810020000001E0E000000003E5A000000803E5C00000000310FAF
:20A9AA0062ED0200120F00000000320FB6A00200130F00000000330FAEA002002310AEA04D
:20A9CA000200271000A00000380F00604200480F01000000280FFEA0020029100000000043
:20A9EA002C0F000000003C0F000042001D0F000000003D0FFDA002002D10AEA002002E10A3
:20AA0A00000000003E0F000000707F0400A000003F0F006042004F0F000043001F1083ED1C
:20AA2A0002000A10ABA0020005105A2F00003E01551C02002406000000855F7000000000D5
:20AA4A00050F5A2500003E01000080955F70000000D87F04000043001F11800000002F0FAA
:20AA6A0000000000050FD5ED02000511B1ED020006109FA002000910A0A002000E10FF2F40
:20AA8A0084013E56CAA00200140F3FC02C003E01791C0200100682EB020008108FC02C00EB
:20AAAA003E01791C02003006000000003E5800A002003E01000080920F70000000007E45B5
:20AACA00000080880F70000000B4AF700000008EDF710000008CFF71080000001E0E882854
:20AAEA0004020122CC2C84831F7101000000060D00C85802012200C858003E018C18888828
:20AB0A007F700000008EDF71000000843F507E1C02003E06000000003F04000000B4AF7055
:20AB2A000000008CFF71010000001E0E000000002090F09F02687F04F92C00C87F04621CC8
:20AB4A0002000206000000787F04000000787F04000000787F04000000787F04D5ED020031
:20AB6A000510509502003E01D5ED020005115E2100003E01601C02000206A3EB0200100FC3
:20AB8A00B6A00200130F85EB0200170F00000000370F00000000390F00000000380F0000C4
:20ABAA0000003D0F00A000003C0F006042004C0F00A000003E0F006042004E0F0000430028
:20ABCA001E1000000000050FD5ED020005119FA002000910A0A002000E10DAA00200120FF8
:20ABEA000DED0200150FFF2F84013E56000000053E5E00300200190F3FC02C003E01C61C9D
:20AC0A0002041006000000017E5A82EB020008108FC02C003E01C61C02003006CDCCCC3D38
:20AC2A000D0F00000000000F000080007E501A0113003E010000008EEF71EAED0200081045
:20AC4A008FC02C003E01B01C020410060000008C9F710000808E9F7100000000010F00007E
:20AC6A0000347E54000000023F50050000001E0E240C13043F58180513023F50C52C08006A
:20AC8A003E01880013863F5A0D1D08003E01400000008014C41C02043A061DA10200001076
:20ACAA00000000400B0FD0408C830F700D0D13003E013D7059003E010D0D13003E013D70C8
:20ACCA0059003E010D0D13003E013D7059003E01070013003E01000000807E500000803FBB
:20ACEA00020F000000003E04000000803E04000000813E5AF09F02487E04F92C00887F0491
:20AD0A009F1C02000206D5ED02000510509502003E01D5ED020005115E2100003E019A1C17
:20AD2A0002000206040000008014591D02003A06B6A00200130F00A00000380F0200430009
:20AD4A00480F000000003C0F000042001D0F000000003E0F000000707F0400A000003F0FAB
:20AD6A00020043004F0F02A043001F1083ED02000A10ACA0020005105A2F00003E01E21C5D
:20AD8A0002002406000000855F7000000000050F5A2500003E01000080955F70000000D89B
:20ADAA007F0402A043001F1100000000050FD5ED02000511B1ED020006109FA002000910F3
:20ADCA00A0A002000E10FF2F84013E5666ED0200120F3FC02C003E01021D0200100682EB3E
:20ADEA00020008108FC02C003E01021D02003006000000003E54000080880F70000000B451
:20AE0A00AF700000008EDF710000008CFF71080000001E0E882804020122CC2C84831F7193
:20AE2A0001000000060D00C85802012200C858003E018C1888887F700000008EDF710000CF
:20AE4A0000843F50071D02003E06000000803E04000000B4AF700000008CFF7101000000D9
:20AE6A001E0E000000002090F09F02687F04F92C00C87F04EE1C02000206000000787F04F1
:20AE8A00000000787F04000000787F04000000787F04D5ED02000510509502003E01D5EDF6
:20AEAA00020005115E2100003E01EC1C0200020643EC0200100FB6A00200130F85EB020064
:20AECA00170F00A000003C0F020043004C0F00A000003E0F020043004E0F02A043001E1015
:20AEEA0000000000050FD5ED020005119FA002000910A0A002000E10D6ED0200150FEAA02D
:20AF0A000200120FFF2F84013E56000000053E5E00340200190F0DED0200150F3FC02C0073
:20AF2A003E014E1D02041006000000017E5A82EB020008108FC02C003E014E1D0200300684
:20AF4A00CDCCCC3D0D0F00000000000F000080007E501A0113003E010000008EEF71EAED9A
:20AF6A00020008108FC02C003E01361D020410060000008C9F710000808E9F7100000000CA
:20AF8A00010F000000347E54000000023F50050000001E0E240C13043F58180513023F5030
:20AFAA00C52C08003E01880013863F5A0D1D08003E011DA1020000104000000080144C1D17
:20AFCA0002043A060000803E0B0F0B0013003E01000000400B0FD0408C830F700D0D1300C7
:20AFEA003E013D7059003E010D0D13003E013D7059003E010D0D13003E013D7059003E0161
:20B00A00070013003E01000000807E500000803F020F000000003E04000000813E5A000054
:20B02A0000803E04F09F02487E04F92C00887F04251D02000206D5ED0200051050950200AD
:20B04A003E01D5ED020005115E2100003E011F1D0200020682EB02000010EAED0200011060
:20B06A00000000043E0A011004003E0182EB020000114BED02000C1020000000040FC42435
:20B08A0000003E01761D02000206000000007E586F12833A010F000080803E58C0AC0C0098
:20B0AA003E01000000400B0FC0408C830F700C0C13003E013C7059003E010C0C13003E0147
:20B0CA003C7059003E010C0C13003E013C7059003E01070013003E011DA1020001101EA18B
:20B0EA0002000410100113003E01140113003E01000000043E0A0000803F040F41220800DD
:20B10A003E01000000043E0A000000017E5A000000000000AAAAAAAA000F9BEB0200001171
:20B12A009CEB020000119DEB02000011EC1D0200BE06AA8C0200001000000000010F012187
:20B14A0000003E01E61D0200000601000000240F00000000340F00005000150F00000000B0
:20B16A00350F00000000380F01000000280F000000003E5B000010103E02A5000000030F52
:20B18A00032000003E01A91D02002006C48C0200140F80000000680FBB1F0200BE06B48C09
:20B1AA000200140F10000000680FBB1F0200BE069DA00200140F80000000680FBB1F020004
:20B1CA00BE061DA10200140F10000000680FBB1F0200BE0600004200180F00600000680F57
:20B1EA00CD1F0200BE0600300200180F00040000680FCD1F0200BE0600340200180F0004AC
:20B20A000000680FCD1F0200BE06D8E60200140FBC000000680FBB1F0200BE062CE3020034
:20B22A00140FAC030000680FBB1F0200BE0614170200BE06AA8C0200001000000000010FD2
:20B24A00012100003E01E61D02000006AA8C0200001002000000010F012100003E01C31DDD
:20B26A00020020060A000000000F928C02000011B08C0200001002000000010F01210000D0
:20B28A003E01BA1D02002006D41D02043E0602000000001401000000001403000000010FED
:20B2AA00012100003E01C01D02002006D41D02043E06020000002014010000000014D41DA7
:20B2CA0002043E06020000000014010000002014AB8C0200001003000000010F1021000042
:20B2EA003E01CA1D0200200601000000000F928C02000011D41D02003E0602000000010F6C
:20B30A00102100003E01D21D020020060A000000000F928C02000011D41D02043E06020015
:20B32A000000201401000000201400000000000F928C02000011AF8C02000010000000000D
:20B34A00010F012100003E01DD1D0200200601000000000F8A8C02000011E61D02043E06CA
:20B36A0000000000000F918C0200001100000000010F8A8C0200011103000000010F012115
:20B38A0000003E01E61D0204000601000000000F918C0200001101000000000F8A8C0200ED
:20B3AA00001100000000000F9BEB020000119CEB020000119DEB02000011EC1D0200BE06C6
:20B3CA00000000003E0A000010000C140A00000000000800ED1D02000E00000000000100BE
:20B3EA00F51D0200000010002C140A00000000000800F61D02000E00000000000100FE1D8E
:20B40A000200000020002C140A00000000001000FF1D02000E00000000000A000F1E020041
:20B42A0000000000000F000008008C14131E02003A0601000000000F9DEB0200031000002B
:20B44A0000000F0F000040002C143FC02C003E01191E02001006000040000C140A00000021
:20B46A0000000800191E02000E00000000000100211E0200000020000C140A0000000000E7
:20B48A000800221E02000E000000000001002A1E0200000020002C140A0000000000100085
:20B4AA002B1E02000E00000000000A003B1E0200000008008C143F1E02003A0600900200EB
:20B4CA003E01009002003E01AA8C02000011000040002C14F09F02003E013FC02C003E014F
:20B4EA00451E02001006000040000C140A00000000000800451E02000E00000000000100E1
:20B50A004D1E0200000020000C140A000000000008004E1E02000E00000000000100561E71
:20B52A000200000020002C140A00000000001000571E02000E00000000000900671E020070
:20B54A0000000000000F000008008C146B1E02003A0601000000000FF09F02003E0100007F
:20B56A0040002C143FC02C003E01701E02001006000040000C140A00000000000800701E31
:20B58A0002000E00000000000100781E0200000020000C140A00000000000800791E02000D
:20B5AA000E00000000000100811E0200000020002C140A00000000001000821E02000E00A7
:20B5CA00000000000A00921E0200000008008C14961E02003A06009002003E0100900200A4
:20B5EA003E01AB8C02000011000040002C14F09F02003E013FC02C003E019C1E020010062C
:20B60A00000040000C140A000000000008009C1E02000E00000000000100A41E020000001F
:20B62A0020000C140A00000000000800A51E02000E00000000000100AD1E020000002000ED
:20B64A002C140A00000000001000AE1E02000E00000000000900BE1E020000000000000FB4
:20B66A00000008008C14C21E02003A0601000000000FF09F02003E01000040002C143FC097
:20B68A002C003E01C71E02001006000040000C140A00000000000800C71E02000E000000D1
:20B6AA0000000100CF1E0200000020000C140A00000000000800D01E02000E000000000040
:20B6CA000100D81E0200000020002C140A00000000001000D91E02000E00000000000A00DC
:20B6EA00E91E0200000008008C14ED1E02003A06009002003E01009002003E01AF8C020063
:20B70A000011000040002C14F09F02003E013FC02C003E01F31E02001006000040000C14CB
:20B72A000A00000000000800F31E02000E00000000000100FB1E0200000020000C140A0066
:20B74A00000000000800FC1E02000E00000000000100041F0200000020002C140A0000001D
:20B76A0000001000051F02000E00000000000900151F020000000000000F000008008C1485
:20B78A00191F02003A0601000000000FF09F02003E01000040002C143FC02C003E011E1F1E
:20B7AA0002001006000040000C140A000000000008001E1F02000E00000000000100261F62
:20B7CA000200000020000C140A00000000000800271F02000E000000000001002F1F020064
:20B7EA00000020002C140A00000000001000301F02000E00000000000A00401F02000000FB
:20B80A0008008C14441F02003A06009002003E01009002003E01B08C0200001100004000A0
:20B82A002C14F09F02003E013FC02C003E014A1F02001006000040000C140A000000000099
:20B84A0008004A1F02000E00000000000100521F0200000020000C140A0000000000080097
:20B86A00531F02000E000000000001005B1F0200000020002C140A000000000010005C1FCA
:20B88A0002000E000000000008006C1F0200821F02003E0604000000680F130000001E0E58
:20B8AA00000040002C14F09F02003E013FC02C003E01741F02001006000040000C140A00AF
:20B8CA00000000000400741F02000E00000000000100781F0200000020000C140A000000D3
:20B8EA0000000400791F02000E000000000001007D1F0200000020002C140A000000000089
:20B90A0004007E1F02000E00000000000900821F0200FFFFFFFF0F0F9CEB020003101400F6
:20B92A000000680F130000001E0E000040002C14F09F02003E013FC02C003E018B1F0200E1
:20B94A001006000040000C140A000000000004008B1F02000E000000000001008F1F0200EE
:20B96A00000020000C140A00000000000400901F02000E00000000000100941F02000000FA
:20B98A0020002C140A00000000000400951F02000E00000000000900991F0200FFFFFFFFAC
:20B9AA000F0F9BEB0200031014000000680F130000001E0E000040002C14F09F02003E01AA
:20B9CA003FC02C003E01A21F02001006000040000C140A00000000000400A21F02000E00DB
:20B9EA00000000000100A61F0200000020000C140A00000000000400A71F02000E00000051
:20BA0A0000000100AB1F0200000020002C140A00000000000400AC1F02000E000000000006
:20BA2A000100B01F0200000010000C140A00000000000400B11F02000E000000000001000B
:20BA4A00B51F0200000010002C140A00000000000400B61F02000E00000000002500BA1FC5
:20BA6A000200000000003E0A100000001E0E000000003E5B000010103E0210F802783E027B
:20BA8A00000000003E5B000010103E02101100003E0111F802783E02000000003E5B0000E7
:20BAAA0010103E02101100003E0111F802783E02000000003E5B000010103E0210110000DF
:20BACA003E0111F802783E02000080803E59000000003E0A100000001E0E000000003E5BA6
:20BAEA00000010103E0210F802783E02000000003E5B000010103E02101100003E0111F8B8
:20BB0A0002783E02000000003E5B000010103E02101100003E0111F802783E020000000045
:20BB2A003E5B000010103E02101100003E0111F802783E02000080803F50000000003E0A08
:20BB4A000800000000005514003002000200000000008A1D00800200050000000000030005
:20BB6A008A9D0200000000100000000000000000000000100000020000000000A0008D9DA6
:20BB8A00020005000000000001002D9E02000000FF3F00000200000000000E002E9E0200AA
:20BBAA0005000000000061023C9E02000000010000000000AC040000000017F90000000076
:20BBCA00AC040000000052BE00000000DCEA000000007D120000000069FF000000007D124F
:20BBEA00000000005FC30000000099DA000000007B2300000000FD0F000000007B2300005E
:20BC0A00000030C5000000005FCA000000000300000000004709000000006AEF0000000050
:20BC2A00470900000000CFDE00000000E7F500000000B41900000000A4E700000000B419FC
:20BC4A000000000079F100000000F0DF000000008A290000000081E9000000008A290000D1
:20BC6A000000DEFD000000004DCD00000000030000000000320D000000002DE7000000006F
:20BC8A00320D00000000C9F2000000002BF900000000D71E000000005AD600000000D71E62
:20BCAA0000000000E30D0000000028E0000000001E2D0000000084D0000000001E2D000098
:20BCCA0000002F1F0000000078CD00000000030000000000C90F000000006BE100000000A0
:20BCEA00C90F00000000D7FD00000000ECF900000000782100000000B5C9000000007821F9
:20BD0A0000000000E51E00000000E7DF000000009F2E000000001BBE000000009F2E0000DD
:20BD2A000000BE330000000000CD00000000030000000000CB11000000003DDD0000000042
:20BD4A00CB1100000000230B00000000E7F900000000692200000000E3C400000000692232
:20BD6A0000000000772B00000000A5E0000000001D2D0000000099B9000000001D2D0000AC
:20BD8A000000F33D0000000095D0000000000300000000001C130000000087DA0000000071
:20BDAA001C1300000000F112000000002BF900000000BF2200000000B6C200000000BF22E9
:20BDCA0000000000B23100000000D4E000000000D32B0000000062B800000000D32B0000AC
:20BDEA000000FD4100000000CBD200000000030000000000491500000000FFD50000000029
:20BE0A0049150000000068190000000007F800000000EC240000000056BC00000000EC2408
:20BE2A000000000089390000000039DF000000007D2D000000001FB1000000007D2D0000FA
:20BE4A0000000B4A000000006CD10000000003000000000091150000000036D50000000092
:20BE6A00911500000000C71B00000000C4F70000000063240000000018BB00000000632494
:20BE8A0000000000C43B0000000001E000000000532C0000000022AF00000000532C0000E9
:20BEAA0000003E4C00000000ADD200000000030000000000351700000000D0D1000000007F
:20BECA00351700000000A2220000000008F600000000D52400000000C8B800000000D524D8
:20BEEA0000000000844000000000A2DF000000007C2B00000000E5AD000000007C2B000013
:20BF0A000000FC4E00000000F1D3000000000300000000007318000000004CCF0000000060
:20BF2A007318000000002F280000000006F400000000A42400000000ACB800000000A42427
:20BF4A0000000000AA42000000007FDF00000000072A00000000B1AF00000000072A0000CB
:20BF6A0000008A4E00000000B6D500000000030000000000711A0000000040CB00000000BB
:20BF8A00711A000000008E2D00000000FFF10000000020260000000015B50000000020260B
:20BFAA000000000018470000000002DE00000000FD2A0000000092AC00000000FD2A0000AC
:20BFCA000000255200000000DBD4000000000300000000003E1A00000000A2CB0000000069
:20BFEA003E1A00000000E52E00000000EAF0000000007A240000000036B8000000007A24C8
:20C00A000000000000450000000021DF0000000071280000000049B10000000071280000A5
:20C02A0000000F4E000000007DD700000000030000000000C71A000000008BCA000000000C
:20C04A00C71A000000000931000000009DEF000000001D2400000000C1B8000000001D2434
:20C06A00000000000F45000000002EDF00000000852700000000C2B2000000008527000089
:20C08A000000F04C0000000071D800000000030000000000D51B0000000067C800000000EF
:20C0AA00D51B00000000B434000000001EED000000008E23000000007DB9000000008E23FB
:20C0CA000000000027450000000034DF00000000152600000000E8B40000000015260000C5
:20C0EA0000003B4B00000000E4D900000000030000000000881C00000000FCC6000000008A
:20C10A00881C00000000F836000000004BEB000000001C23000000002FBA000000001C23A6
:20C12A0000000000E344000000003FDF000000001625000000008EB60000000016250000F6
:20C14A000000CE4900000000DFDA00000000030000000000B71E0000000098C200000000D3
:20C16A00B71E00000000303C00000000BFE700000000FE230000000043B800000000FE2391
:20C18A0000000000374700000000E3DD000000005B2500000000B6B5000000005B250000EC
:20C1AA000000E04A000000008CDA00000000030000000000E51E0000000038C200000000E5
:20C1CA00E51E00000000F73C0000000082E600000000372300000000B4B900000000372396
:20C1EA0000000000F4450000000056DE000000003A2400000000CAB7000000003A2400008B
:20C20A000000DD4800000000A5DB000000000300000000004C1C0000000068C700000000D5
:20C22A004C1C0000000043380000000012E700000000EC1E0000000034C200000000EC1E0E
:20C24A0000000000A93D0000000004E200000000611F0000000054C100000000611F0000F3
:20C26A000000533F0000000070E000000000030000000000381D000000008FC50000000026
:20C28A00381D00000000413A000000005FE500000000381F0000000098C100000000381F79
:20C2AA0000000000553E000000007CE100000000741F0000000024C100000000741F000079
:20C2CA0000008C3F0000000052E000000000030000000000270D00000000A0190000000067
:20C2EA00270D00000000840400000000BFFA00000000241C000000002E2F00000000241CE2
:20C30A000000000002E700000000B6E400000000B82700000000E63A00000000B8270000B2
:20C32A00000094D300000000ABD300000000030000000000080800000000DE0E000000000F
:20C34A0008080000000082250000000024F500000000FD1500000000DB1900000000FD15EB
:20C36A0000000000D11100000000F1E1000000009D2400000000A61C000000009D240000BB
:20C38A00000081030000000006CF000000000300000000003905000000001D0900000000D3
:20C3AA0039050000000096360000000070EF00000000F01000000000770C00000000F01087
:20C3CA0000000000602B00000000E0DF00000000411F00000000950700000000411F0000AD
:20C3EA000000F92300000000B6CE00000000030000000000570500000000510900000000DA
:20C40A00570500000000CD370000000012EF00000000501100000000BE0C00000000501125
:20C42A0000000000572C0000000029DF00000000F31F00000000C00700000000F31F00007C
:20C44A000000C624000000009DCD000000000300000000003D0300000000950400000000A2
:20C46A003D0300000000CB4900000000A7E600000000360E0000000019FE00000000360E32
:20C48A0000000000304700000000CCD900000000431D0000000092ED00000000431D000037
:20C4AA00000092470000000060CB000000000300000000009D020000000054030000000075
:20C4CA009D0200000000AE51000000008CE200000000E90C00000000E2FA00000000E90C80
:20C4EA000000000013510000000000D700000000B81B000000000AE800000000B81B00005F
:20C50A000000485300000000ABC9000000000300000000003A02000000007C020000000045
:20C52A003A0200000000F9560000000083DF000000003A0C000000005AF8000000003A0C26
:20C54A0000000000BA5700000000E5D400000000F81A0000000093E300000000F81A00006D
:20C56A000000145B000000008BC8000000000300000000000C0200000000D301000000000A
:20C58A000C0200000000015B0000000024DD000000009D0C00000000F9F4000000009D0CE7
:20C5AA0000000000FF5C00000000E0D200000000141C000000001BDD00000000141C00000C
:20C5CA00000036610000000059C700000000030000000000980100000000F7000000000007
:20C5EA00980100000000B96100000000D3D800000000770B0000000014F300000000770BC8
:20C60A0000000000A0640000000012D0000000006D1A0000000028DA000000006D1A00001A
:20C62A0000007C69000000000CC6000000000300000000006B010000000056000000000074
:20C64A006B010000000060650000000027D600000000CB0B00000000F7EF00000000CB0B10
:20C66A000000000000690000000028CE000000004B1B000000008FD4000000004B1B000022
:20C68A000000176E0000000058C5000000000300000000003F0100000000000000000000AB
:20C6AA003F0100000000CD6800000000BCD300000000600B000000002BEF00000000600B7C
:20C6CA00000000008C6C000000008FCC00000000AD1A000000005ED300000000AD1A00003E
:20C6EA0000009671000000009EC4000000000300000000001B0100000000BCFF00000000ED
:20C70A001B0100000000566B00000000BED100000000050B0000000093EE00000000050B02
:20C72A0000000000156F0000000054CB000000001C1A0000000092D2000000001C1A00007C
:20C74A000000EF73000000003BC40000000003000000000013010000000079FF00000000DF
:20C76A00130100000000096D0000000060D000000000720B00000000ECEC00000000720B23
:20C78A0000000000DD70000000005BCA00000000F21A00000000A5CF00000000F21A000091
:20C7AA0000008A7500000000E1C300000000030000000000CA000000000070FF0000000090
:20C7CA00CA00000000002871000000002BCD00000000620900000000B1EF0000000062097E
:20C7EA00000000005974000000008AC80000000010170000000085D5000000001017000068
:20C80A0000007E78000000002CC300000000030000000000E70000000000F5FE000000004C
:20C82A00E70000000000A4730000000042CB00000000780B00000000DCEA00000000780B17
:20C84A0000000000FA7600000000E7C600000000191B000000005FCC00000000191B00001E
:20C86A000000BB7A0000000056C2000000000300000000009600000000003AFF000000008F
:20C88A00960000000000D4760000000070C8000000004E080000000060F0000000004E087A
:20C8AA00000000003379000000007DC500000000E71400000000A6D700000000E71400000D
:20C8CA000000367C00000000FDC100000000030000000000130200000000130200000000B1
:20C8EA00000000000000843B00000000000000000000CB0300000000F9F800000000CB03E2
:20C90A0000000000CD780000000050C600000000AE0F000000009AE100000000AE0F0000BD
:20C92A0000005A7C000000005AC20000000003000000000084000000000018FF000000005D
:20C94A00840000000000407B000000009FC40000000013080000000029F0000000001308DC
:20C96A0000000000C37C00000000EFC200000000481400000000DFD700000000481400004F
:20C98A000000F77D0000000042C100000000030000000000BE000000000096FE00000000C1
:20C9AA00BE0000000000657C0000000088C300000000240B00000000E4E900000000240B58
:20C9CA0000000000BA7D000000001AC2000000002B1A00000000E6CB000000002B1A0000FF
:20C9EA0000003A7E0000000015C10000000003000000020000000000B70B9DA00200050094
:20CA0A0000000000010054AC0200000064A10200020000000000F10A55AC020005000000FD
:20CA2A000000010046B70200000056AC0200020000000000F12047B70200050000000000D0
:20CA4A00010038D80200000048CD0200020000000000F10A39D8020005000000000001008C
:20CA6A002AE30200000048CD02000200000000006E082BE30200050000000000020099EB73
:20CA8A00020000000100000000000100000002000000000029029BEB0200050000000000CE
:20CAAA000B00C4ED02006E0083F9A23E0000001049405D007A7715B7000000008035FD007F
:20CACA0038774FABBD00AA72302F8C00A531D7B2EF001BEF3836CD00000D50B9890088889D
:20CAEA00083CAB00AAAA2ABE0200000000001E00CFED0200080000000000FCFF00004200DE
:20CB0A000800000000000400FCFF42000C00000000000100000043000000006042000800C8
:20CB2A000000000001A0010043000C0000000000020002A0430000000200430000000000CE
:20CB4A000000000000000000000000003E0B00000000000000000000000000000000000082
:20CB6A000000000000000020802D73395B1602003E06000000003E0B000000003E0B0000E9
:20CB8A0000000000000000000000000000000000000000000000000000003E0B0000000042
:20CBAA003E0B000000003E0B000000003E0B000000003E0B000000003E0B000000003E0BB5
:20CBCA00000000003E0B000000003E0B000000003E0B000000003E0B000000003E0B0000DE
:20CBEA0000003E0B000000003E0B000000003E0B000000003E0B000000003E0B00000000BE
:20CC0A003E0B000000003E0B000000003E0B85000200BE06000000003E0B000000003E0B52
:20CC2A00000000003E0B0000000000000000000000000000000000000000000000000000A1
:20CC4A0000003E0B000000003E0B000000003E0B000000003E0B88070200BE060000000051
:20CC6A003E0B000000003E0B000000003E0B000000003E0B000000003E0B000000003E0BF4
:20CC8A00000000003E0B000000003E0B000000003E0B000000003E0B000000003E0B00001D
:20CCAA0000003E0B000000003E0B000000003E0B000000003E0B000000003E0B00000000FD
:20CCCA003E0B000000003E0B000000003E0B000000003E0B000000003E0B000000003E0B94
:20CCEA00000000003E0B000000003E0B000000003E0B000000003E0B000000003E0B0000BD
:20CD0A0000003E0B000000003E0B000000003E0B000000003E0B000000003E0B000000009C
:20CD2A003E0B000000003E0B000000003E0B000000003E0B000000003E0B000000003E0B33
:20CD4A00000000003E0B000000003E0B000000003E0B000000003E0B000000003E0B00005C
:20CD6A0000003E0B000000003E0B000000003E0B000000003E0B000000003E0B000000003C
:20CD8A003E0B000000003E0B000000003E0B000000003E0B000000003E0B000000003E0BD3
:20CDAA00000000003E0B000000003E0B000000003E0B000000003E0B000000003E0B0000FC
:20CDCA0000003E0B000000003E0B000000003E0B000000003E0B000000003E0B00000000DC
:20CDEA003E0B000000003E0B000000003E0B000000003E0B000000003E0B000000003E0B73
:20CE0A00000000003E0B000000003E0B000000003E0B000000003E0B000000003E0B00009B
:20CE2A0000003E0B000000003E0B000000003E0B000000003E0B000000003E0B000000007B
:20CE4A003E0B000000003E0B000000003E0B000000000000000000000000000000000000ED
:20CE6A00000000000000000000000000000400000B14800000000B14080000000B1420009F
:20CE8A0000000B14100000000B14008002007C1100000000000F338C02000011328C02008A
:20CEAA000110101102003E015004020000064AED02000010009002003E014AED0200001135
:20CECA0001000000240FFFFFFFFF250F010000002C0F000000003C0F928C020001100A0022
:20CEEA000000000F012000003E01B40002002006BB8C0200001000940C003E0102000000A3
:20CF0A008014A90002003A0684ED02000110109102003E0184ED02000111110300003E0249
:20CF2A00412000003E01A9000200220600000004001400000000010F928C02000111B40066
:20CF4A0002003E06010000008014B40002003A0686ED02000110109102003E0186ED020019
:20CF6A000111110300003E02412000003E01B4000200220600000004001400000000010F9B
:20CF8A00928C0200011100000000340F40410000010F01007000011100000000000F0010DF
:20CFAA0002003E01C1000204000641EB0200140F163802001C0F01000000000F001002006B
:20CFCA003E01C100020020064BEB0200140F203802001C0FE1FFFFFF0C0FCDCCCC3D040F91
:20CFEA00FFFFFFFF0F0FB0ED020003100A000000680F0A0000001E0E000070000110111002
:20D00A0001003E021CA00D003E0100020B003E01042208003E01D0000204020600000080A6
:20D02A003F59F09F02003E013F032C003E01000000803E59B0ED0200031140410000010F76
:20D04A00010070000111AAAA0000000F00007000001158EB0200140F2D3802001C0F000065
:20D06A000000000F09000000680F020000001E0E000000803F59000000803E5900000000BA
:20D08A00000F001002003E01E3000200000601000000000F001002003E0139010200000698
:20D0AA0000000000000F57EB020000112C38020000130180020000118A8C020000100010BD
:20D0CA0002003E012101020000068B8C02000010001002003E01FA00020000062F8C0200A2
:20D0EA0000102C8C02000410041008003E01F40002000206DB0FC940040F042008003E017E
:20D10A002F8C02000011F9160204BE062F8C02000011000000000000B78C02000110010039
:20D12A0013003E010180020000118C8C02000010001002003E010B0102000006308C0200B2
:0ED14A0000102D8C02000410041008003E019D
:00000001FF
